:020000040000FA
:04000000B3EF15F055
:08000800F2EF15F0186E7F0BFA
:1000100018BC8008F76A240FF66E0800F55018BE69
:1000200000081200000306090C101316191C1F22E9
:1000300025282B2E313336393C3F414447494C4E1D
:10004000515355585A5C5E60626466686A6B6D6FA6
:1000500070717374757678797A7A7B7C7D7D7E7E1B
:100060007E7F7F7F7F002C6A2D6A01D0206E215019
:10007000205ED8A021062D502C5ED8A02D06D89049
:1000800021322032D8902D322C32031C1C6E041CDD
:100090001D6E1C2AD8B41D2A830E276E286A296A71
:1000A0002A6A2B6A266A0F0EEA6E02C0E9FF091C53
:1000B000D5EC02F000D000D0040020502826D8B0A3
:1000C000292A215029262C502A26D8B02B2A2D50F7
:1000D0002B2629509BDF800F196E2B5097DF800F46
:1000E00019261930262602C0E9FFEF500910D8A0C2
:1000F0000918EF6E2704D8B4830E276ED8B41C2AD3
:10010000D8B41D3ED7D71200086A800E346E89EF2E
:1001100000F0206A216A226A236A0A9AF2EC01F04E
:10012000D30FD8B40A8A2D0FC60FF8E20A0FF6E3F0
:100130001C6E1B6A1A6A196A0A0E186EB3EC02F07A
:100140001C501824206E1950216E000ED8B0010EDC
:1001500021261A50226E000ED8B0010E22261B5006
:10016000236E000ED8B0010E2326080606E0F2EC3E
:1001700001F0C60F02E20A0FDBE20AAA0BD0201E32
:10018000211E221E231E202AD8B4212AD8B4222AB6
:10019000D8B4232A20501200086A206E216A0096E3
:1001A0000850D8B40086050E076E270E1D6E100E7F
:1001B0000CD8030E1D6EE80E08D81D6A640E05D813
:1001C0001D6A0A0E02D8205008D01C6E2150196EEC
:1001D0002050186E9CEC02F01850186E074E0096D6
:1001E000085003E0075CD8B008D01850D8A4009697
:1001F00000B603D0300FE5EF01F01200366E2DAEE1
:1002000003D02D0EE5EC01F0106A116A126A136A30
:100210002D8E6A0E2C26D8902D322E322F3213328C
:100220001232113210322C3EF6D72F502C5C2F2672
:100230002C5E2E502D5C2E262D5E086A3AD82E0E8E
:10024000E5EC01F0376AD89010342F6E11342E6E21
:1002500012342D6E13342C6E3736D8902F362E363E
:100260002D362C36373610502F261150D8B0113C71
:100270002E261250D8B0123C2D261350D8B0133C65
:100280002C26D8B0373ED8902F362E362D362C3629
:1002900037363750300FE5EC01F02FC010F02EC08C
:1002A00011F02DC012F02CC013F0362ECBD7D89001
:1002B00012000096085003E100860A0E086E2FC057
:1002C0001BF02EC01AF02DC019F02CC018F0076AD0
:1002D000236A226A216A0A0E206E3FEC02F0072A86
:1002E0000750085CD8A4F4D72050D8A4009600A6E4
:1002F00002D0082C04D02050300FE5EC01F0082E7D
:10030000DED71200206E0750D8B4120020C0E9FFDB
:1003100021C0EAFFEF50D8B41200E5EC01F0204A0A
:10032000212A0706F0D7246E0F0EEA6EE26E025005
:10033000E96E120FE16E800E0A16080E256ED89037
:10034000D8B00A3E12D82432252EFAD7000029BA96
:100350000A300BD800D000D000D0D88006D8065084
:100360001D6E055025EC02F0120029AE0BD0EF50A7
:10037000091029AC0918EF6EE7500910D8A0091828
:10038000E76E0AD0EF500910D8A0091829BC091847
:10039000EF6E091CE71600D029501F0B000F196ED5
:1003A0002850110FD8B0192A000032EF02F0A66AC7
:1003B000A68E0900F55002E002D8FBD71200040017
:1003C0009EA8FDD7AD6ED880120001BA93EF01F060
:1003D00001B4DFEF01F001A205D001B003D001B2FA
:1003E000EE6E120034BEEE501200AA6AA96EA66A22
:1003F000A680A850A94AAA2A1200AA6AA86EA66ACC
:10040000A684550EA76EAA0EA76EA6820400A6B2F9
:10041000FDD7A694A94AAA2A1200E836E8363C0B72
:100420000109C212C009C216C050F80B0209C06E01
:10043000320E31EC02F0C2820400C2B2FDD7C4CF4A
:100440002DF0C3502C6E12001D6A1C6EFF0E1C2670
:100450001D2200D0D8A01200030E196EE70E02D89C
:10046000F5D7196AFD0F186EFF0E00D001D01826BF
:10047000040000D0D8A01926D8A01200F8D71B502D
:100480002318800BF46E1BAE06D0D880000E1856D1
:1004900019561A561B5623AE06D0D880000E205689
:1004A0002156225623561C6A1D6A1E6A1F6A306A2C
:1004B000316A326A336A235022102110201023E05F
:1004C000200EF36ED890183619361A361B36303691
:1004D0003136323633362050305C2150315822507C
:1004E00032582350335809E32050305E2150315A9E
:1004F0002250325A2350335AD8801C361D361E36AD
:100500001F36F32EDFD7F4AE06D0D880000E1C566F
:100510001D561E561F561CC018F01DC019F01EC0D7
:100520001AF01FC01BF030C020F031C021F032C0E3
:1005300022F033C023F01200216A206A100EF36EFD
:100540001934203621361C50205C1D50215805E3FB
:100550001C50205E1D50215AD88018361936F32EB3
:10056000EFD718501200200E246E306A316A326ABA
:10057000336AD89018A00ED0205030262150D8B021
:10058000213C31262250D8B0223C32262350D8B00C
:10059000233C332633323232313230321B321A327C
:1005A00019321832242EE5D71200E988E92AEC1610
:1005B0001200A66AA68E0900F55002E0EE6EFBD787
:1005C0001200F34E02D0E652FCD7E6CFEEFFE82E43
:1005D000FCD71200E466FED7F36EE552F32EFDD78A
:1005E000E6CFEEFFE82EFCD71200610EE75C05E6D1
:1005F0007B0EE75C02E7DF0EE716E650EE6EF5E1F4
:100600001200A66AA68EEE500900F55C02E1F566BE
:10061000FAD71200155011183A6E3ABE30D015BEF6
:1006200017D01450105CD8A0000CD8A4010C1550A1
:10063000115CD8A0000CD8A4010C1650125CD8A0F4
:10064000000CD8A4010C1750135CD8A0000C010CAE
:100650001050145CD8A0000CD8A4010C1150155CEB
:10066000D8A0000CD8A4010C1250165CD8A0000C25
:10067000D8A4010C1350175CD8A0000C010C11AECB
:10068000010C000C155011183A6E3ABE34D015BE4C
:1006900019D01450105CD8A0000CD8A4010C15502F
:1006A000115CD8A0000CD8A4010C1650125CD8A084
:1006B000000CD8A4010C1750135CD8A0000CD8A4CF
:1006C000010C000C1050145CD8A0000CD8A4010C34
:1006D0001150155CD8A0000CD8A4010C1250165C67
:1006E000D8A0000CD8A4010C1350175CD8A0000CA3
:1006F000D8A4010C000C11AE010C000C1450105CBD
:10070000376E19E2376C10C039F014C010F039C0E0
:1007100014F011C039F015C011F039C015F012C035
:1007200039F016C012F039C016F013C039F017C0F6
:1007300013F039C017F01A0E376078D0145276E0F3
:10074000366A1150396E15183B6E118E158E080ED3
:10075000375E08E317C036F016C017F015C016F064
:10076000156AF5D7372607E0D890153216321732BA
:100770003632372EF9D73BAE35D01750135E1650B0
:10078000125A1550115A07E2D880000E135612560D
:100790001156800E391A366C04E01306000E125AF8
:1007A000115A040E376E11660DD012C011F013C02D
:1007B00012F036C013F0366A080E105E2DE3372EA5
:1007C000F2D72AD011BE08D0D8903636133612365A
:1007D0001136102EF7D720D038AC26D036AE24D024
:1007E000366A11D0175013261650122215501122B6
:1007F00006E31132123213323632104A0FD038ACBF
:1008000013D036AE11D0133E0FD0123E0DD0113E94
:100810000BD0D8801390EDD7106A02D038821068C0
:10082000136A126A800E116E39AE119E13501200B7
:100830001150326E15183B6E145053E0105254E0B4
:10084000105E7F0E03E2102603E24DD010264EE22A
:1008500013C030F012C031F0328E158E180E396E82
:10086000136A126A116A0BD01750305C1650315857
:1008700011E3316E326A1750305E0BD004E215502E
:10088000325CF2E007E31750305E1650315A1550D3
:10089000325AD88013361236113630363136323667
:1008A000392EECD711BE07D010521DE03B32100696
:1008B000392A3B36E3D738AC1FD007E21750305EF9
:1008C0001650315A1550325A17E3133E15D0123EC6
:1008D00013D0113E11D0113212321332103E0CD00F
:1008E00005D0388604D03884106A02D03882106867
:1008F000136A126A800E116E3BAE119E13501200E5
:100900001150326E15183B6E1050D8A414503CE0B4
:1009100010267E0E03E3105E03E338D0105E33E34F
:1009200013C030F012C031F0328E158E136A126A85
:10093000116A180E396E32323132303206E31750F6
:100940001326165012221550112211321232133270
:10095000392EF1D711BE07D0133612361136105288
:1009600012E01006323438AC17D016E3133E14D020
:10097000123E12D0113E10D0D880113212321332F2
:10098000103E0AD003D03884106A02D03882106832
:10099000136A126A800E116E3BAE119E1350120044
:1009A000126A136A10C036F013C010F036C013F08C
:1009B00012C036F011C012F036C011F0960E396E2A
:1009C0003B6A10AE07D0D880000E1356125611564F
:1009D00010563B8E105218E038AC0DD013AE0BD031
:1009E000123E09D0113E07D0103E05D0D8801032FB
:1009F00011321232392A080E392612C013F011C0F2
:100A000012F010C011F015D0116613D0080E395E27
:100A1000125005E1080E395E135011E0136A116E91
:100A200013C012F0136A05D0D8901336123611365F
:100A3000390611AEF9D739C010F03BAE119E1350F4
:100A400012003D3D3D3D3D3D3D3D3D3D3D3D3D3D3E
:100A50003D3D3D3D3D3D3D3D3D3D3D3D3D3D3D3DC6
:100A60003D3D3D3D3D3D3D3D3D004E657720435084
:100A70005520636869702064657465637465642ECD
:100A800000003D3D3D3D3D3D3D3D3D3D3D3D3D3D10
:100A90003D3D3D3D3D3D3D3D3D3D3D3D3D3D3D3D86
:100AA0003D3D3D3D3D3D3D3D3D003D3D3D3D3D3DB3
:100AB0003D3D3D3D3D3D3D3D3D3D3D3D3D3D3D3D66
:100AC0003D3D3D3D3D3D3D3D3D3D3D3D3D3D3D3D56
:100AD0003D0053696572726120526164696F2053F1
:100AE000797374656D732054522053657175656E0A
:100AF000636572004669726D776172652076657212
:100B000073696F6E20002C206275696C6420000090
:100B10004E6574776F726B206164647265737320C5
:100B20002000456E746572202F2F68656C702066FA
:100B30006F7220636F6D6D616E642073756D6D6192
:100B4000727900003D3D3D3D3D3D3D3D3D3D3D3DDE
:100B50003D3D3D3D3D3D3D3D3D3D3D3D3D3D3D3DC5
:100B60003D3D3D3D3D3D3D3D3D3D3D00456E74655A
:100B70007220636F6D6D616E642000002F2F6F75A2
:100B8000743033206F6E00004641494C00004865C8
:100B90007921206E657720636F6D6D616E64000052
:100BA0006E65745F7061636B65742073686F756CDC
:100BB0006420626520636C656172203C00006E6594
:100BC000745F7061636B65745F6C656E203D2000BF
:100BD0007061636B6574203D20006E65745F73798E
:100BE0006E633D006E65745F747970653D006E657F
:100BF000745F66726F6D3D006E65745F746F3D006B
:100C00006E65745F6372633D00006E65745F706152
:100C1000796C6F61643D3C006E65745F7061636BFD
:100C200065745F6C656E3D006E65745F7061796CB4
:100C30006F61645F6C656E3D00002E2E2E20636830
:100C400065636B2074686520435243202E2E2E006E
:100C50006C656E677468206F6620617267203D2046
:100C6000000043616C63756C61746564204352439A
:100C7000203D20002C205061636B6574204352435B
:100C8000203D2000435243204661696C65642E205C
:100C900020426164207061636B657400435243209D
:100CA00050617373656420212020476F6F6420506A
:100CB00061636B6574006D79206164647265737340
:100CC0003D00484559212074686973207061636B49
:100CD000657420697320666F72206D6521004E6F08
:100CE00074206D79206164647265737300005365CC
:100CF0006E643A20000053656E643A20000053652C
:100D00006E643A20000053656E643A20000049206A
:100D10006861766520746865206E6574776F726BA4
:100D200020286E65745F61737365727420616374EB
:100D30006976652900004E6574776F726B20726565
:100D40006C656173656400004E6F77206174207478
:100D5000686520657865637574655F6E65745F634B
:100D60006F6D6D616E642073746570006E65745F85
:100D70007061636B65745F6C656E3D3D00002020A3
:100D8000636D645F64656C696D3D3D002020636D3B
:100D9000645F64656C696D3D3D3D0000636D645F3B
:100DA00064656C696D20203D0000636D645F636F56
:100DB0006D6D616E643D0000636D645F61726720FC
:100DC0002020203D00004F504D4F444500004F4E25
:100DD00044454C41593100004F4E44454C41593235
:100DE00000004F4E44454C41593300004F4E44459E
:100DF0004C41593400004F4E44454C415935000098
:100E00004F464644454C415931004F464644454CB7
:100E1000415932004F464644454C415933004F46F4
:100E20004644454C415934004F464644454C41598F
:100E30003500454E41424C45000044495341424C27
:100E400045004E4F524D414C4F4E00004F6E2073A7
:100E5000657175656E6365203D206E6F726D616CA6
:100E60000000524556455253454F4E004F6E207379
:100E7000657175656E6365203D2072657665727378
:100E800065004E4F524D414C4F4646004F6666201E
:100E900073657175656E6365203D206E6F726D615F
:100EA0006C00524556455253454F464600004F662A
:100EB000662073657175656E6365203D2072657689
:100EC0006572736500004F55543031004F555430F2
:100ED00032004F55543033004F55543034004F5585
:100EE00054303500494E3100494E3200494E3300EE
:100EF00050554C534500435700004B4559004B4556
:100F00005945520057504D004556454E543100004A
:100F10004556454E543200004556454E5433000068
:100F20004556454E543400004556454E5435000054
:100F30004556454E543600004556454E5437000040
:100F4000574D0000574D4C494D4954004144314DD7
:100F5000494E00004144324D494E00004144334D5A
:100F6000494E00004144344D494E00004144314D4A
:100F7000415800004144324D415800004144334D36
:100F8000415800004144344D415800004144414C17
:100F900041524D00414443414C31000041444341E2
:100FA0004C320000414443414C3300004144434132
:100FB0004C340000534554524556000053455442AA
:100FC00055494C4400004E4554004C4F43414C00A1
:100FD00048454C5000004C4F414400005341564599
:100FE000000053544154555300005354415445009C
:100FF000555044415445000044454255474F4E002A
:101000004465627567206D6F6465204F4E004445EE
:101010004255474F464600004465627567206D6F34
:101020006465204F46460000535244454255474FA1
:101030004E005368696674207265676973746572DF
:10104000206465627567206D6F6465204F4E0000F7
:10105000535244454255474F46460000536869661F
:101060007420726567697374657220646562756760
:10107000206D6F6465204F4646004E4554444542FE
:1010800055474F4E00004E6574776F726B20646554
:10109000627567206D6F6465204F4E004E45544465
:1010A000454255474F4646004E6574776F726B2038
:1010B0006465627567206D6F6465204F4646000069
:1010C00050494E470000524F4C4C43414C4C00009D
:1010D000464F5243454641494C0045594543414ED0
:1010E00044590000455945004D5347444952454332
:1010F0005400536574206D657373616765206D6F6F
:10110000646520746F206469726563742E004D53AA
:10111000474E45540000536574206D6573736167D5
:1011200065206D6F646520746F206E6574776F72D3
:101130006B207061636B6574206D6F64652E0000B9
:101140004543484F00005354415445545249474782
:10115000455200005245534554005245424F4F54AA
:1011600000004745544144445200534554414444CF
:1011700052005241440053494C454E5400004D4FDB
:1011800044450000424F4F5400002050494E473A1A
:1011900020002C2046726F6D3A2000002C20416404
:1011A00064726573733A20005354415445313A00D8
:1011B0005354415445313A005354415445313A0057
:1011C0005354415445323A005354415445333A0044
:1011D0005354415445343A005354415445353A0030
:1011E0005354415445313A005354415445323A0026
:1011F0005354415445333A005354415445343A0012
:101200005354415445353A0055504441544500002B
:101210004F4B000053595354454D204641494C2CE7
:101220002066726F6D3A20002E202053687574740A
:10123000696E6720646F776E2E005365742050438B
:1012400020757064617465207472696767657220C7
:10125000746F2000435720444F4E45004F4E00000E
:101260004B65796572206D6F6465204F4E004B654C
:10127000796572206D6F6465204F464600005365A6
:101280007420435720737065656420746F200000DC
:1012900053656E642043573A20002D2D2D2D2D20AF
:1012A000412F4420434F4E564552544552205641FB
:1012B0004C554553202D2D2D2D2D2D2D2D2D000040
:1012C000416E616C6F6720696E2031203D20000007
:1012D00076202046776420202800416E616C6F677D
:1012E00020696E2032203D20000076202052656665
:1012F00020202800416E616C6F6720696E203320CA
:101300003D20000076202020202020202800416E53
:10131000616C6F6720696E2034203D2000007620CC
:1013200020202020202028002D2D2D2D2D2D2D2D6D
:101330002D2D2D2D2D2D2D2D2D2D2D2D2D2D2D2DDD
:101340002D2D2D2D2D2D2D2D2D2D2D2D00004F4EE4
:101350000000416E616C6F6720696E70757420616A
:101360006C61726D206D6F6465204F4E00004F46BA
:101370004600416E616C6F6720696E707574206104
:101380006C61726D206D6F6465204F464600536539
:101390007420412F442031206D696E696D756D2078
:1013A000746F200053657420412F442032206D69F2
:1013B0006E696D756D20746F200053657420412F28
:1013C000442033206D696E696D756D20746F200047
:1013D00053657420412F442034206D696E696D750A
:1013E0006D20746F200053657420412F44203120FC
:1013F0006D6178696D756D20746F20005365742080
:10140000412F442032206D6178696D756D20746FB5
:10141000200053657420412F442033206D6178698A
:101420006D756D20746F200053657420412F44202A
:1014300034206D6178696D756D20746F200053657F
:101440007420412F4420696E7075742031206361CF
:101450006C6962726174696F6E2076616C7565206B
:10146000746F200053657420412F4420696E70759D
:101470007420322063616C6962726174696F6E20DE
:1014800076616C756520746F200053657420412F60
:101490004420696E70757420332063616C696272D8
:1014A0006174696F6E2076616C756520746F2000C1
:1014B00053657420412F4420696E70757420342068
:1014C00063616C6962726174696F6E2076616C75BC
:1014D0006520746F2000212121204C6F7720766FCA
:1014E0006C7461676520616C61726D206F6E20693C
:1014F0006E7075742023302E20204D696E203D20A3
:101500000000762E202041637475616C203D200020
:10151000212121204C6F7720766F6C7461676520E4
:10152000616C61726D206F6E20696E70757420231E
:10153000312E20204D696E203D200000762E202087
:1015400041637475616C203D2000212121204C6F86
:101550007720766F6C7461676520616C61726D20B5
:101560006F6E20696E7075742023322E20204D69B5
:101570006E203D200000762E202041637475616C42
:10158000203D2000212121204C6F7720766F6C7444
:1015900061676520616C61726D206F6E20696E708D
:1015A00075742023332E20204D696E203D200000CD
:1015B000762E202041637475616C203D200021212E
:1015C00021204F76657220766F6C746167652061AB
:1015D0006C61726D206F6E20696E7075742023309F
:1015E0002E20204D6178203D2000762E2020416362
:1015F0007475616C203D2000212121204F76657299
:1016000020766F6C7461676520616C61726D206F0C
:101610006E20696E7075742023312E20204D617804
:10162000203D2000762E202041637475616C203DA2
:101630002000212121204F76657220766F6C746125
:10164000676520616C61726D206F6E20696E7075C8
:10165000742023322E20204D6178203D2000762EEC
:10166000202041637475616C203D200021212120E0
:101670004F76657220766F6C7461676520616C616E
:10168000726D206F6E20696E7075742023332E206A
:10169000204D6178203D2000762E20204163747516
:1016A000616C203D20004F46460057617474206DE8
:1016B000657465722070726F74656374696F6E20F3
:1016C00064697361626C656400004F4E00004261A2
:1016D0007369632077617474206D6574657220701E
:1016E000726F74656374696F6E20656E61626C659C
:1016F0006400435553544F4D0000456E61626C6564
:10170000207573657220646566696E656420776113
:101710007474206D657465722070726F7465637483
:10172000696F6E2072616E6765004B657920696E26
:1017300070757420676F657320696E616374697674
:1017400065004B657920696E70757420676F6573ED
:10175000206163746976650053494C454E5400001E
:10176000564552424F534500426F6F7420696E20B8
:10177000766572626F7365206D6F646500004F4E11
:10178000000053696C656E74206D6F6465204F4670
:1017900046004C4F43414C004E4554574F524B006E
:1017A00043616C6C207369676E2073657420746F7D
:1017B0002000536574206669726D776172652072CE
:1017C000657620746F200000536574206669726D21
:1017D00077617265206275696C6420746F20000007
:1017E0004E6574776F726B206164647265737320E9
:1017F00073657420746F2000536574206D79206EBA
:101800006574776F726B20616464726573732074A2
:101810006F200000536574205478204F4E2064657B
:101820006C6179203120746F2000536574205478E6
:10183000204F4E2064656C6179203220746F200047
:10184000536574205478204F4E2064656C61792074
:101850003320746F2000536574205478204F4E203D
:1018600064656C6179203420746F200053657420A6
:101870005478204F4E2064656C6179203520746F58
:1018800020005365742052782064656C61792031A2
:1018900020746F2000005365742052782064656CBA
:1018A0006179203220746F200000536574205278D3
:1018B0002064656C6179203320746F2000005365CB
:1018C000742052782064656C6179203420746F2014
:1018D00000005365742052782064656C617920356E
:1018E00020746F2000004F7574707574200020659F
:1018F0006E61626C656400004F75747075742000D1
:101900002064697361626C6564004F4E00004F464D
:1019100046005475726E206F757470757420312096
:101920004F4E00005475726E206F75747075742080
:1019300031204F4646004F4E00004F46460054753A
:10194000726E206F75747075742032204F4E0000D7
:101950005475726E206F75747075742032204F4606
:1019600046004F4E00004F4646005475726E206F81
:1019700075747075742033204F4E00005475726E6C
:10198000206F75747075742033204F4646004F4E9B
:1019900000004F4646005475726E206F7574707566
:1019A000742034204F4E00005475726E206F757491
:1019B0007075742034204F4646004F4E00004F464D
:1019C00046005475726E206F7574707574203520E2
:1019D0004F4E00005475726E206F757470757420D0
:1019E00035204F4646004F4E00004F464600547586
:1019F000726E20696E7075742031204F4E005475E0
:101A0000726E20696E7075742031204F464600005A
:101A10004F4E00004F4646005475726E20696E703E
:101A200075742032204F4E005475726E20696E70AE
:101A300075742032204F464600004F4E00004F463E
:101A400046005475726E20696E7075742033204F95
:101A50004E005475726E20696E7075742033204F7D
:101A600046460000526573657420616C6C2070619D
:101A700072616D657465727320746F206465666150
:101A8000756C742076616C7565732E00436F6E669D
:101A9000696775726174696F6E2073617665642021
:101AA000746F20666C617368206D656D6F72792E3E
:101AB0000000436F6E66696775726174696F6E20AE
:101AC0006C6F616465642066726F6D20666C617313
:101AD00068206D656D6F72792E002D2D2D2054526A
:101AE00020537175656E63657220436F6D6D616E15
:101AF0006473202D2D2D2D2D2D2D2D2D2D2D2D2DA6
:101B00002D2D2D2D2D2D2D2D2D2D2D2D2D2D2D2D05
:101B10002D2D2D2D2D004F4E44454C4159306E201A
:101B20007820206D732E2044656C61792078202800
:101B3000312D3530303029206D732E206265666F6F
:101B40007265207475726E696E67206F6E206F7596
:101B50007470757420236E2C202077686572652060
:101B60006E203D20312D35004F464644454C4159AD
:101B7000306E2078206D732E2044656C617920785A
:101B80002028312D3530303029206D732E206265AC
:101B9000666F7265207475726E696E67206F666617
:101BA000206F757470757420236E2C2077686572B1
:101BB00065206E203D20312D35004E4F524D414C59
:101BC0004F4E2020202020202020205475726E208F
:101BD0006F6E2020696E206E6F726D616C202073B5
:101BE000657175656E63652C20312C20322C203395
:101BF0002C20342C203520202844656661756C74B7
:101C000029004E4F524D414C4F4646202020202067
:101C10002020205475726E206F666620696E206EDB
:101C20006F726D616C202073657175656E63652CD4
:101C300020352C20342C20332C20322C2031202015
:101C40002844656661756C742900524556455253A7
:101C5000454F4E20202020202020205475726E20D9
:101C60006F6E2020696E20726576657273652073D1
:101C7000657175656E63652C20352C20342C2033FE
:101C80002C20322C20310000524556455253454FEE
:101C90004646202020202020205475726E206F663A
:101CA0006620696E20726576657273652073657152
:101CB00075656E63652C20312C20322C20332C204E
:101CC000342C20350000454E41424C4520782020E0
:101CD00020202020202020456E61626C6573206FDB
:101CE000757470757420782028312D352900444989
:101CF0005341424C452078202020202020202044A1
:101D0000697361626C6573206F7574707574207887
:101D10002028312D352900002D2D2D2041646D699D
:101D20006E20436F6D6D616E6473202D2D2D2D2DF2
:101D30002D2D2D2D2D2D2D2D2D2D2D2D2D2D2D2DD3
:101D40002D2D2D2D2D2D2D2D2D2D2D2D2D2D2D2DC3
:101D50002D2D2D2D000048454C50202020202020E6
:101D600020202020202020446973706C6179207429
:101D70006869732068656C7020696E666F726D614A
:101D800074696F6E00005354415455532020202035
:101D900020202020202020446973706C61792074F9
:101DA00068652063757272656E7420636F6E666914
:101DB0006775726174696F6E00004C4F414420205A
:101DC00020202020202020202020204C6F61642013
:101DD000636F6E66696775726174696F6E20667293
:101DE0006F6D20666C617368206D656D6F72790030
:101DF0005341564520202020202020202020202034
:101E0000205361766520636F6E66696775726174D1
:101E1000696F6E20746F20666C617368206D656DEC
:101E20006F727900524553455420202020202020F5
:101E300020202020205265736574206F70657261C8
:101E400074696E6720706172616D6574657273206C
:101E5000746F207374616E6461726420646566617E
:101E6000756C742076616C75657300005245424F45
:101E70004F54202020202020202020202052656246
:101E80006F6F74207468652073797374656D0000DA
:101E9000424F4F542053494C454E5420202020207F
:101EA000205475726E73206F666620626F6F7420A7
:101EB0006D65737361676500424F4F5420564552FC
:101EC000424F534520202020205475726E73206F9E
:101ED0006E20626F6F74206D6573736167650000BB
:101EE00053544154455452494747455220787878D5
:101EF00020557064617465732050432070726F6761
:101F000072616D20646973706C6179206966206408
:101F1000656C6179206973203E2078787820286488
:101F2000656661756C74203D20323530206D7329F3
:101F300000002D2D2D20412F4420436F6E766572B9
:101F4000746572202D20416E616C6F6720496E7040
:101F500075742043616C6962726174696F6E2D2DB6
:101F60002D2D2D2D2D2D2D2D2D2D2D2D2D2D0000FB
:101F7000414443414C6E2078787820202020202056
:101F800020416473206F7220737562747261637490
:101F90007320746865206F6666736574207878783E
:101FA0002028696E206D696C69766F6C74732920C6
:101FB000746F2074686520412F4420636F6E7665CE
:101FC0007274657220276E27202028312D34290055
:101FD00041446E4D494E20787878202020202020E2
:101FE0002053657473206C6F77207472696767651E
:101FF0007220616C61726D20766F6C746167652010
:10200000746F2078787820766F6C74732028696EEE
:1020100020766F6C7473290041446E4D41582078CE
:102020007878202020202020205365747320686950
:102030006768207472696767657220616C61726D90
:1020400020766F6C7461676520746F2078787820D3
:10205000766F6C74732028696E20766F6C747329A8
:102060000000524144202020202020202020202039
:102070002020205265616420616E616C6F67206969
:102080006E70757420766F6C74616765206E6F7703
:1020900000002D2D2D2057617474204D65746572DC
:1020A00020436F6D6D616E6473202D2D2D2D2D2DB0
:1020B0002D2D2D2D2D2D2D2D2D2D2D2D2D2D2D2D50
:1020C0002D2D2D2D2D2D2D2D2D2D2D2D2D2D00009A
:1020D000574D204F4E20202020202020202020203F
:1020E000205475726E206F6E206261736963207771
:1020F000617474206D65746572206D6F6E69746FA4
:1021000072696E672E202048696768207265666C68
:10211000656374656420706F7765722064697361AC
:10212000626C65732073657175656E63657200001E
:10213000574D204F464620202020202020202020C0
:10214000205475726E206F66662062617369632029
:1021500077617474206D65746572206D6F6E69743B
:102160006F72696E672E0000574D20435553544FD0
:102170004D20202020202020205475726E206F6E6C
:102180002077617474206D65746572206D6F6E695F
:10219000746F72696E672E2020496E686962697477
:1021A0002073657175656E6365207768656E207252
:1021B00065666C656374656420766F6C74616765D1
:1021C00020686974732074686520574D4C494D49E7
:1021D000542076616C756500574D4C494D4954202B
:1021E0007878782020202020204D696E696D756DEB
:1021F000207265666C656374656420766F6C7461CB
:10220000676520746861742077696C6C20696E68FA
:1022100069626974207468652073657175656E63A1
:1022200065002D2D2D2054524947474552204556D3
:10223000454E54532D2D2D2D2D2D2D2D2D2D2D2D48
:102240002D2D2D2D2D2D2D2D2D2D2D2D2D2D2D2DBE
:102250002D2D2D2D2D2D2D2D2D2D2D2D2D2D000008
:102260004F504D4F44452078787820202020202062
:1022700020536574206F7065726174696E67206D9C
:102280006F64653A203120646972656374207374E9
:102290006174696F6E20636F6E74726F6C20286456
:1022A000656661756C7429206F722032205452204B
:1022B00053657175656E636572206D6F64650000AE
:1022C0004556454E543120782020202020202020C3
:1022D00020536574206576656E7420312E2E2E3362
:1022E00020746F206D6F646520312070756C73658C
:1022F0002C2032206F6E2C2033206F66662C203409
:102300002073656E64207570646174652C203520BF
:10231000746F67676C6500002D2D2D204357204397
:102320006F6D6D616E6473202D2D2D2D2D2D2D2D36
:102330002D2D2D2D2D2D2D2D2D2D2D2D2D2D2D2DCD
:102340002D2D2D2D2D2D2D2D2D2D2D2D2D2D2D2DBD
:102350002D2D2D2D00004B45594552204F4E20204C
:10236000202020202020205475726E206F6E206B5C
:1023700065796572206D6F64652E20204F757470CD
:10238000757420352077696C6C2073656E6420430A
:1023900057207573696E6720746865204357206302
:1023A0006F6D6D616E6400004B45594552204F467C
:1023B0004620202020202020205475726E206F6639
:1023C00066206B65796572206D6F64652E20204FE5
:1023D000757470757420352077696C6C206F70652A
:1023E0007261746520696E206E6F726D616C20730E
:1023F000657175656E636572206D6F646500435726
:1024000020787878787820202020202020202053E1
:10241000656E64207465787420787878787820699F
:102420006E204357207573696E67206F75747075E1
:1024300074203520696E206B65796572206D6F643C
:10244000650057504D207878202020202020202023
:1024500020202053657420435720737065656420E5
:10246000696E20617070726F78696D617465207734
:102470006F72647320706572206D696E757465206B
:1024800028312D39392900002D2D2D204E657477E6
:102490006F726B20436F6D6D616E6473202D2D2DF7
:1024A0002D2D2D2D2D2D2D2D2D2D2D2D2D2D2D2D5C
:1024B0002D2D2D2D2D2D2D2D2D2D2D2D2D2D2D2D4C
:1024C0002D2D2D2D00005345544144445220787841
:1024D00020202020202020576865726520787820F1
:1024E00069732074686520626F6172642773206E5F
:1024F0006574776F726B20616464726573732028F2
:102500006265747765656E203120616E64203135B7
:1025100029004745544144445220202020202020B7
:10252000202020476574207468652076616C75658D
:10253000206F662074686520626F61726427732063
:102540006E6574776F726B2061646472657373007B
:1025500053494C454E54204F4E202020202020200F
:1025600020446F206E6F742073656E64206D6573F8
:10257000736167657320746F2073657269616C2085
:10258000706F7274207768656E2073746174652053
:102590006368616E6765730053494C454E54204F24
:1025A00046462020202020202053656E64206D6543
:1025B00073736167657320746F2073657269616CF2
:1025C00020706F7274207768656E20737461746513
:1025D000206368616E67657300004D53474449523C
:1025E0004543542020202020202020536574207251
:1025F0006573706F6E736520746F20706C61696EA7
:10260000207465787420666F726D617400004D539C
:10261000474E4554202020202020202020202053D9
:10262000657420726573706F6E736520746F206EB1
:102630006574776F726B207061636B657420666F71
:10264000726D617400002D2D2D204D616E75616CD1
:10265000204F757470757420436F6D6D616E647377
:10266000202D2D2D2D2D2D2D2D2D2D2D2D2D2D2DA7
:102670002D2D2D2D2D2D2D2D2D2D2D2D2D2D2D2D8A
:102680002D2D00004F5554306E204F4E202020201D
:1026900020202020204D616E75616C6C792074754E
:1026A000726E204F4E20206F7574707574206E20EE
:1026B00028312D3529004F5554306E204F46462085
:1026C000202020202020204D616E75616C6C7920C7
:1026D0007475726E204F4646206F75747075742045
:1026E0006E2028312D3529002D2D2D20496E746541
:1026F000726E616C20446562756767696E6720431E
:102700006F6D6D616E6473202D2D2D2D2D2D2D2D52
:102710002D2D2D2D2D2D2D2D2D2D2D2D2D2D2D2DE9
:102720002D2D2D2D000044454255474F4E20202091
:10273000202020202020205475726E206F6E20648F
:102740006562756767696E67206D6573736167653C
:10275000730044454255474F464620202020202004
:102760002020205475726E206F6666206465627545
:102770006767696E67206D657373616765730000D5
:10278000464F5243454641494C20202020202020DE
:1027900020466F7263657320756E697420696E746C
:1027A0006F204641494C206D6F64652E2020536890
:1027B000757473206F666620616C6C206F75747021
:1027C000757473003D3D3D3D3D5B20435552524580
:1027D0004E5420434F4E46494755524154494F4E5F
:1027E000205D3D3D3D3D3D3D3D3D3D00436F6E66C1
:1027F000696720636F646520203A2000426F617230
:102800006420747970652020203A20004657207695
:10281000657273696F6E2020203A2000465720624F
:1028200075696C6420202020203A20004D792061B9
:102830006464726573732020203A20004F4E20207C
:1028400064656C6179203120203A20004F4E2020B1
:1028500064656C6179203220203A20004F4E2020A0
:1028600064656C6179203320203A20004F4E20208F
:1028700064656C6179203420203A20004F4E20207E
:1028800064656C6179203520203A20004F4646204F
:1028900064656C6179203120203A20004F46462043
:1028A00064656C6179203220203A20004F46462032
:1028B00064656C6179203320203A20004F46462021
:1028C00064656C6179203420203A20004F46462010
:1028D00064656C6179203520203A20003A20456EED
:1028E00061626C6564003A2044495341424C45445E
:1028F00000004F7574707574203120202020200056
:102900003A20456E61626C6564003A204449534147
:10291000424C454400004F7574707574203220207D
:10292000202020003A20456E61626C6564003A20E8
:1029300044495341424C454400004F7574707574CE
:1029400020332020202020003A20456E61626C65F3
:1029500064003A2044495341424C454400004F75BD
:102960007470757420342020202020003A20456E99
:1029700061626C6564003A2044495341424C4544CD
:1029800000004F75747075742035202020202000C1
:102990004F4E2073657175656E636520203A204E39
:1029A0006F726D616C004F4E2073657175656E635B
:1029B0006520203A205265766572736564004F4643
:1029C000462073657175656E6365203A204E6F729F
:1029D0006D616C004F46462073657175656E636569
:1029E000203A205265766572736564004357207300
:1029F0007065656420202020203A2000576174749F
:102A0000206D6574657220636865636B696E67200D
:102A10004F46460053696D706C6520776174742071
:102A20006D6574657220636865636B696E672065A8
:102A30006E61626C6564000057617474206D65742A
:102A40006572206C696D69742073657420746F20E1
:102A50000000414420616C61726D206D6F64653AC5
:102A6000204F66660000414420616C61726D206DEC
:102A70006F64653A204F4E00416E616C6F67203184
:102A8000206D696E203A2000202020202020202068
:102A9000206D6178203A2000202020202020202056
:102AA0002063616C203A2000416E616C6F672032B8
:102AB000206D696E203A2000202020202020202038
:102AC000206D6178203A2000202020202020202026
:102AD0002063616C203A2000416E616C6F67203387
:102AE000206D696E203A2000202020202020202008
:102AF000206D6178203A20002020202020202020F6
:102B00002063616C203A2000416E616C6F67203455
:102B1000206D696E203A20002020202020202020D7
:102B2000206D6178203A20002020202020202020C5
:102B30002063616C203A2000436F6D6D206D6F64DF
:102B400065202020203A204C6F63616C0000436FA9
:102B50006D6D206D6F6465202020203A204E6574D5
:102B6000776F726B0000F86A400E386E006A030ED1
:102B7000AF6E200EAC6E900EAB6E2EEE81F0949880
:102B80008298949A829A939081909392819293944E
:102B90008194110E05012F6FC70E2E6F510E2D6FF0
:102BA000810E2C6F0101D99DD98F040E196EB00EC4
:102BB000186E1D6A91C51CF09CEC02F005018F6F28
:102BC00019C090F5030E8E6F520E8D6F05EEE4F076
:102BD000540EEE6E520EEE6E310EEE6EEF6A000186
:102BE00029EF16F09EAA23D0060EAB141DE1E2CF0A
:102BF0003DF0E1CF3CF03E2AFF0E3E5C01E33E6A31
:102C00001DEE82F03E50E126000EE222AECFE7FF3D
:102C10000D0EE75C02E1010E426E3EC018F43DC0AD
:102C2000E2FF3CC0E1FF1100AB98AB8800D011007F
:102C30003E6A3F6A9D8AC00EF26E12009D9A0DEEAA
:102C400082F0FF0EEE6AE82EFDD73E6A3F6A9D8A4B
:102C50001200400EAF6E900EAB6E200EAC6E0B0EDF
:102C6000C16EF19E320E24EC02F08298829A81901D
:102C70008192819493948194939281929390819084
:102C8000949A829A949882980101D99BD9BF8282A2
:102C9000D9AF829205012B910101CC6BD46BDB6B18
:102CA000DA6B01EEDCF04F0EEE6E4B0EEE6EEF6A5D
:102CB000010EE16F01EE1CF0EE6A01EEE2F0EE6A49
:102CC0000401A16B640EA06FA36BA26B04EE1AF05B
:102CD000300EEE6EEE6EEF6A06011189118B119DBA
:102CE0000401A46B04EEA5F0EE6A0501286B276BC6
:102CF000EE89EE8BEE8DEE8F0601118111930501A9
:102D0000786BCD0E7C6FCC0E7B6F4C0E7A6F7C0E89
:102D1000796F0601119511970101686B6A6B0501C6
:102D2000266B4B6B4A6B496B486B4F6B4E6B4D6B15
:102D30004C6B536B526B516B506B576B566B556BA7
:102D4000546B01016B6B05015B6B5A6B596B586BD4
:102D50005F6B5E6B5D6B5C6B636B626B616B606B1F
:102D6000676B666B656B646B6B6B6A6B700E696F20
:102D7000830E686F6F6B6E6B700E6D6F830E6C6F72
:102D8000736B726B700E716F830E706F776B766BF7
:102D9000700E756F830E746F01016C6B49DF00015B
:102DA000FEEC18F00101D991D993D995010E0501D6
:102DB000EB6F010EDF6FE16B050EE06FE36B050E4D
:102DC000E26F010EED6F5B6B5A6B596B586B6B6B5F
:102DD0006A6B200E696F810E686F5F6B5E6B5D6B57
:102DE0005C6B6F6B6E6B200E6D6F810E6C6F636B27
:102DF000626B616B606B736B726B200E716F810E17
:102E0000706F676B666B656B646B776B766B200EB0
:102E1000756F810E746FEE972A6B640E296FEB2924
:102E2000EC6F0001CEEC2BF082B618EF17F0F9D75B
:102E300094908280000EF5EC01F00501DF6FDF2930
:102E40000001D8A44FEF17F00401A4530001D8A447
:102E50004FEF17F004EEA5F00A0EF76E420EF66E75
:102E6000D9EC02F0EF6AF9EC1EF004EEA5F00A0EC0
:102E7000F76E6A0EF66ED9EC02F0EF6AF9EC1EF00E
:102E8000B0EC46F05EEC47F004EEA5F00A0EF76EEB
:102E9000820EF66ED9EC02F0EF6AF9EC1EF0D2EC7D
:102EA0004AF01FEC3AF001EE6DF0020E016E0501E2
:102EB000ED51CCEC00F0EF6A010E0401A453D8A44C
:102EC000000E356E010E01016B53D8A4000E3514AF
:102ED0000001D8B4E1EF17F004EEA5F00A0EF76E8A
:102EE000AA0EF66ED9EC02F0EF6AF9EC1EF004EED1
:102EF000A5F00A0EF76ED20EF66ED9EC02F0EF6A6C
:102F0000F9EC1EF004EEA5F00A0EF76EF40EF66E64
:102F1000D9EC02F0020E016E086AE1C521F0E0C5AD
:102F200020F0CFEC00F00B0EF76E060EF66ED9EC2B
:102F300002F0020E016E086AE3C521F0E2C520F03E
:102F4000CFEC00F0EF6AF9EC1EF004EEA5F00B0EEA
:102F5000F76E100EF66ED9EC02F0020E016E05014E
:102F6000ED51CCEC00F0EF6A04EEA5F00B0EF76E1D
:102F7000220EF66ED9EC02F0EF6A0001F9EC1EF0B9
:102F800004EEA5F00B0EF76E440EF66ED9EC02F0CF
:102F9000EF6AF9EC1EF004EEA5F00B0EF76E6C0E66
:102FA000F66ED9EC02F0EF6AF9EC1EF004EEA5F033
:102FB0000B0EF76E7C0EF66ED9EC02F0EF6ADFECCA
:102FC0001EF0320E24EC02F0949082900B0EF76EFD
:102FD000880EF66E01EEDCF001EC03F0D8A4F3EFFE
:102FE00017F02FEC2CF0D896060111ADD886000111
:102FF000D8B6FDEF17F032EF18F001EEA0F0020E98
:10300000016EE86A80BA010ECCEC00F0EF6A01EEC6
:10301000A0F084EC00F0808AE8A0809A01EEB5F080
:10302000020E016EE86A81B6010ECCEC00F0EF6A88
:1030300001EEB5F084EC00F08186E8A0819641ECC9
:1030400031F0010E01016C5D0001D8A42AEF18F0E7
:1030500003EC37F0050178530001D8B432EF18F0D3
:10306000AAEC39F00601119D010E0101E15D00019C
:10307000D8A43DEF18F0ADEF18F0020E0101E15DAC
:103080000001D8A446EF18F048EF18F0BEEF18F092
:1030900081A84DEF18F0ABEF18F0010E0101CC6FD5
:1030A000E86A80BA010E356EE86A81B6010E351005
:1030B0000001D8B461EF18F00101CC6B000164EF9E
:1030C00018F0010E0101CC6F0001010E0101CC5D71
:1030D000010ED8A4000E356E010E05012BBDE86A65
:1030E00035140001D8B477EF18F02BEF41F0010E42
:1030F0000101CC5D010ED8A4000E356EE86A050111
:103100002BBD010E35140001D8B489EF18F09EEFE5
:103110003BF0010E0101CC53D8A4000E356E010E18
:1031200005012BBDE86A35140001D8B49AEF18F0F8
:103130006CEF3EF0010E0101CC53D8A4000E356EA9
:10314000E86A05012BBD010E35140001D8B4ABEFC0
:1031500018F030EF41F0BEEF18F080AAB2EF18F08F
:1031600030EC3AF081A6B7EF18F069EC3AF081A89C
:10317000BCEF18F0A2EC3AF0BEEF18F00501274BB7
:10318000282B2751295D28512A590001D8B0E7EF93
:1031900018F00501286B276BD8962BB1D886000153
:1031A000D8B6DAEF18F005012B81949282920001D3
:1031B000E7EF18F0D89605012BA1D8860001D8B604
:1031C000E6EF18F005012B91949282820001040130
:1031D000A251A05DA351A1590001D8B0F5EF18F09C
:1031E000FEEC18F00401A36BA26B0001010E425C1F
:1031F000D8A4FDEF18F002EC19F0E8D6426A1EECF4
:1032000016F01200D8960101D9A5D8860001D8B6CB
:1032100016EF19F00B0EF76E8E0EF66ED7EC01F06E
:103220000D0EDFEC01F00A0EDFEC01F001EEE2F032
:10323000820EEE6AE82EFDD7D8960101D9A5D88670
:103240000001D8B63AEF19F00B0EF76EA00EF66E2D
:10325000D7EC01F001EEE2F0EE5003E0DFEC01F01C
:10326000FBD73E0EDFEC01F00D0EDFEC01F00A0E95
:10327000DFEC01F03E040401186F00013EAE43EFA5
:1032800019F00401186B0001D8960101D9A5D88660
:103290000001D8B65EEF19F00B0EF76EBE0EF66E9B
:1032A000D7EC01F0040E016E04011851CCEC00F0D3
:1032B0000D0EDFEC01F00A0EDFEC01F0000104015D
:1032C00018530001D8A468EF19F0010E0401186F1B
:1032D0000001040118050B6E0101CC6B0001010116
:1032E000CC510B5C0001D8A0AEEF19F0D8960101CB
:1032F000CCAFD8860001D8B680EF19F00101CC6BB5
:1033000000010101CC290DEE82F0E926000EEA222F
:10331000EFCF0FF001EEE2F0CC51E926000EEA22E9
:103320000FC0EFFFD896D9A5D8860001D8B6A8EF70
:1033300019F0040E016E01EEE2F00101CC51E92614
:10334000000EEA22EF50CCEC00F0200EDFEC01F092
:1033500000010101CC2B0001D8A4C0D7B1EC19F0B9
:10336000120001EEE2F011EEE2F0F5EC02F0D89678
:103370000101D9A5D8860001D8B6D2EF19F00B0EFD
:10338000F76ED00EF66ED7EC01F001EEE2F0EE50E3
:1033900003E0DFEC01F0FBD70D0EDFEC01F00A0ECD
:1033A000DFEC01F002EE64F011EEE2F0010EF36EDC
:1033B000010EE1EC02F0EF6AD8960101D9A5D8869A
:1033C0000001D8B6F7EF19F00B0EF76EDA0EF66EB5
:1033D000D7EC01F002EE64F0EE5003E0DFEC01F018
:1033E000FBD70D0EDFEC01F00A0EDFEC01F002EE70
:1033F00066F011EEE2F0020EF36E010EE1EC02F067
:10340000EF6AD8960101D9A5D8860001D8B61CEF7D
:103410001AF00B0EF76EE40EF66ED7EC01F002EE2A
:1034200066F0EE5003E0DFEC01F0FBD70D0EDFECB1
:1034300001F00A0EDFEC01F002EE69F011EEE2F0AD
:10344000030EF36E020EE1EC02F0EF6AD896010172
:10345000D9A5D8860001D8B641EF1AF00B0EF76E49
:10346000EE0EF66ED7EC01F002EE69F0EE5003E0DE
:10347000DFEC01F0FBD70D0EDFEC01F00A0EDFEC04
:1034800001F002EE6DF011EEE2F0050EF36E020EA9
:10349000E1EC02F0EF6AD8960101D9A5D8860001C7
:1034A000D8B666EF1AF00B0EF76EF80EF66ED7EC84
:1034B00001F002EE6DF0EE5003E0DFEC01F0FBD71F
:1034C0000D0EDFEC01F00A0EDFEC01F002EE71F000
:1034D00011EEE2F0070EF36E030EE1EC02F0EF6A7C
:1034E000D8960101D9A5D8860001D8B68BEF1AF07D
:1034F0000C0EF76E000EF66ED7EC01F002EE71F0D6
:10350000EE5003E0DFEC01F0FBD70D0EDFEC01F035
:103510000A0EDFEC01F002EE76F011EEE2F00A0E98
:10352000F36E090E0401185DE1EC02F0EF6AD89623
:103530000101D9A5D8860001D8B6B5EF1AF00C0E56
:10354000F76E0A0EF66ED7EC01F002EE76F0EE5052
:1035500003E0DFEC01F0FBD73E0EDFEC01F00D0ED7
:10356000DFEC01F00A0EDFEC01F001EEE2F0E86AB8
:10357000EE5202E0E83EFCD70401186FD896010134
:10358000D9A5D8860001D8B6D8EF1AF00C0EF76E80
:10359000180EF66ED7EC01F0040E016E04011851FE
:1035A000CCEC00F00D0EDFEC01F00A0EDFEC01F0C8
:1035B000000102EE76F0E86AEE5202E0E83EFCD747
:1035C0000401196FD8960101D9A5D8860001D8B693
:1035D000FCEF1AF00C0EF76E280EF66ED7EC01F029
:1035E000040E016E04011951CCEC00F00D0EDFEC5D
:1035F00001F00A0EDFEC01F0000104EE1AF012EE09
:1036000069F0030EE75204E0E6CFEEFFE82EFAD7AA
:10361000EF6A300E0201665D0001D8A412EF1BF0C4
:10362000B6EF1CF02F0E0201665D0001D8A41BEF5F
:103630001BF00101D98B00012F0E0201665D000114
:10364000D8A428EF1BF004EE1AF0300EEE6EEF6AED
:103650002F0E0201665D0001D8A431EF1BF083EC50
:1036600020F02F0E0201665D0001D8A43DEF1BF093
:1036700001016A6B000140EF1BF0010E01016A6F4E
:1036800000012F0E0201665D0001D8A449EF1BF076
:103690001200D8960101D9A5D8860001D8B65DEFF1
:1036A0001BF00C0EF76E3A0EF66ED7EC01F00D0E15
:1036B000DFEC01F00A0EDFEC01F0D8960101D9A58C
:1036C000D8860001D8B677EF1BF00C0EF76E500EBF
:1036D000F66ED7EC01F0040E016E0101D451CCEC72
:1036E00000F00D0EDFEC01F00A0EDFEC01F000013E
:1036F0000401176B010E0101CC6F0001060E0101E0
:10370000CC5D0001D8B0E1EF1BF001EEE2F0010169
:10371000CC51E926000EEA22EF50D46FD4510401B7
:10372000171B01EEA0F0020E016E0101CC51CCEC92
:1037300000F0EF6A01EEB5F0020E016E04011751C0
:10374000CCEC00F0EF6AD8960101D9A5D88600012B
:10375000D8B6DBEF1BF001EEA0F0EE5003E0DFEC9B
:1037600001F0FBD7200EDFEC01F001EEE2F00101E9
:10377000CC51E926000EEA22EF50DFEC01F0200EDA
:10378000DFEC01F0630EDFEC01F0720EDFEC01F014
:10379000630EDFEC01F03D0EDFEC01F001EEB5F061
:1037A000EE5003E0DFEC01F0FBD70D0EDFEC01F093
:1037B0000A0EDFEC01F000010101CC2B0001D8A4BE
:1037C0009CD7090E0101CC6F00010101CC5104010D
:1037D000185D0001D8A049EF1CF001EEE2F00101F4
:1037E000CC51E926000EEA22EF500B6E0B5004017B
:1037F000171B01EEA0F0020E016E0101CC51CCECC2
:1038000000F0EF6A01EEB5F0020E016E04011751EF
:10381000CCEC00F0EF6AD8960101D9A5D88600015A
:10382000D8B643EF1CF001EEA0F0EE5003E0DFEC61
:1038300001F0FBD7200EDFEC01F001EEE2F0010118
:10384000CC51E926000EEA22EF50DFEC01F0200E09
:10385000DFEC01F0630EDFEC01F0720EDFEC01F043
:10386000630EDFEC01F03D0EDFEC01F001EEB5F090
:10387000EE5003E0DFEC01F0FBD70D0EDFEC01F0C2
:103880000A0EDFEC01F000010101CC2B0001D8A4ED
:103890009BD7D8960101D9A5D8860001D8B670EF7C
:1038A0001CF00C0EF76E620EF66ED7EC01F0040EF3
:1038B000016E04011751CCEC00F00C0EF76E740E83
:1038C000F66ED7EC01F002EE71F0EE5003E0DFECA3
:1038D00001F0FBD70D0EDFEC01F00A0EDFEC01F07A
:1038E000000102EE71F084EC00F00B6E21C00CF0D0
:1038F00022C00DF023C00EF00D500E100AE10C5046
:103900000D1007E10B50040117190001D8B4A2EF04
:103910001CF0D8960101D9A5D8860001D8B69DEF34
:103920001CF00C0EF76E840EF66ED7EC01F00D0E47
:10393000DFEC01F00A0EDFEC01F0FEEC18F01200F3
:10394000B6EF1CF0D8960101D9A5D8860001D8B6EB
:10395000B6EF1CF00C0EF76E9C0EF66ED7EC01F075
:103960000D0EDFEC01F00A0EDFEC01F0D89601013C
:10397000D9A5D8860001D8B6D0EF1CF00C0EF76E92
:10398000B60EF66ED7EC01F0040E016E0501ED5196
:10399000CCEC00F00D0EDFEC01F00A0EDFEC01F0D4
:1039A000000102EE6DF084EC00F00101D46FD76BE2
:1039B000D4510501ED5D0001D8A4E2EF1CF0010E29
:1039C0000101D76F0001630E0101D45D0001D8A48D
:1039D000EDEF1CF0010E0101D76F0001630E010134
:1039E000D45D0001D8A4F8EF1CF0020E01016A6F4B
:1039F0000001010E0101D75D0001D8A41EEF1DF0EA
:103A0000D8960101D9A5D8860001D8B614EF1DF0CB
:103A10000C0EF76EC20EF66ED7EC01F00D0EDFEC59
:103A200001F00A0EDFEC01F002EE76F012EE76F015
:103A3000F5EC02F09AEC20F032EF1DF0D89601017F
:103A4000D9A5D8860001D8B632EF1DF00C0EF76E5E
:103A5000DE0EF66ED7EC01F00D0EDFEC01F00A0E73
:103A6000DFEC01F0FEEC18F0120002EECBF011EEEC
:103A700031F0360EE75204E0E6CFEEFFE82EFAD73B
:103A8000EF6A46EC1DF0EEEC1FF0120003EE0DF0B5
:103A9000820EEE6AE82EFDD702EEB8F02F0EEE6E23
:103AA000EF6A02EEBBF0410EEE6EEF6A02EEBEF080
:103AB000020E016E0501ED51CCEC00F0EF6A02EE52
:103AC000BEF0E86AEE5202E0E83EFCD70B6E010E53
:103AD0000B5C0001D8A47DEF1DF001EEB5F0300EB7
:103AE000EE6E12EEBEF0030EE75204E0E6CFEEFFFC
:103AF000E82EFAD7EF6A89EF1DF001EEB5F012EE6D
:103B0000BEF0030EE75204E0E6CFEEFFE82EFAD750
:103B1000EF6A02EEBEF011EEB5F0140EE75204E0CB
:103B2000E6CFEEFFE82EFAD7EF6A02EEC2F014EE0F
:103B30001AF0030EE75204E0E6CFEEFFE82EFAD7C4
:103B4000EF6A02EEC2F0E86AEE5202E0E83EFCD70D
:103B50000101D46FD4530001D8A4B5EF1DF002EEDB
:103B6000C2F0300EEE6EEE6EEF6A010E0101D45D12
:103B70000001D8A4D6EF1DF004EEA5F0300EEE6ED5
:103B800012EEC2F0030EE75204E0E6CFEEFFE82E9D
:103B9000FAD7EF6A02EEC2F014EEA5F0800EE752FB
:103BA00004E0E6CFEEFFE82EFAD7EF6A020E01013D
:103BB000D45D0001D8A4E3EF1DF002EEC2F0EE5098
:103BC000FEE1ED52EF6A01EE6DF012EEB8F0020E7A
:103BD000E75204E0E6CFEEFFE82EFAD712EEBBF094
:103BE000020EE75204E0E6CFEEFFE82EFAD712EE1F
:103BF000BEF0030EE75204E0E6CFEEFFE82EFAD760
:103C000012EEC2F0030EE75204E0E6CFEEFFE82E1C
:103C1000FAD712EECBF0410EE75204E0E6CFEEFF0A
:103C2000E82EFAD7EF6A01EE6DF0E86AEE5202E094
:103C3000E83EFCD70101D86FD76B01EE6DF0E86A62
:103C4000EE5202E0E83EFCD70B6E010ECC6F000195
:103C50000101CC510B5C0001D8A04BEF1EF001EE2E
:103C60006DF00101CC51EB50D46FD451D71B01EE54
:103C7000A0F0020E016ECC51CCEC00F0EF6A01EE28
:103C8000B5F0020E016ED751CCEC00F0EF6ACC2BF0
:103C90000001D8A4DCD702EEC6F0020E016E0101CD
:103CA000D751CCEC00F0EF6A02EEC6F0E86AEE52B3
:103CB00002E0E83EFCD7D46F010ED45D0001D8A429
:103CC00071EF1EF004EEA5F0300EEE6EEE6E12EE09
:103CD000C6F0040EE75204E0E6CFEEFFE82EFAD776
:103CE000EF6A020E0101D45D0001D8A486EF1EF038
:103CF00004EEA5F0300EEE6E12EEC6F0040EE752A2
:103D000004E0E6CFEEFFE82EFAD7EF6A030E0101DA
:103D1000D45D0001D8A499EF1EF004EEA5F012EED8
:103D2000C6F0040EE75204E0E6CFEEFFE82EFAD725
:103D3000EF6A02EEC6F014EEA5F0800EE75204E042
:103D4000E6CFEEFFE82EFAD7EF6A03EE0DF012EEA3
:103D5000B8F0020EE75204E0E6CFEEFFE82EFAD705
:103D600012EEBBF0020EE75204E0E6CFEEFFE82EC3
:103D7000FAD712EEBEF0030EE75204E0E6CFEEFFF4
:103D8000E82EFAD712EEC2F0030EE75204E0E6CFB7
:103D9000EEFFE82EFAD712EEC6F0040EE75204E06A
:103DA000E6CFEEFFE82EFAD712EECBF0410EE75247
:103DB00004E0E6CFEEFFE82EFAD7EF6A1200800E9D
:103DC000026E100E096E400E296E540E286E066AA1
:103DD000056A200E016E810E076E040E216EA50E7F
:103DE00082EC01F00D0E93EC01F00A0E93EC01F061
:103DF000120001016A530001D8A447EF1FF023EC21
:103E000020F0D8960101D9A5D8860001D8B61CEFBC
:103E10001FF00C0EF76EEE0EF66ED7EC01F004EE0E
:103E2000A5F0EE5003E0DFEC01F0FBD70D0EDFEC68
:103E300001F00A0EDFEC01F00401A4530001D8A444
:103E40002FEF1FF004EEA5F0EE5003E0DFEC01F0E1
:103E5000FBD70D0EDFEC01F00A0EDFEC01F0010ED6
:103E60000401A45D0001D8A443EF1FF004EEA5F007
:103E7000EE5003E0DFEC01F0FBD70D0EDFEC01F0BC
:103E80000A0EDFEC01F06CEC20F0EDEF1FF0010EFC
:103E900001016A5D0001D8A496EF1FF023EC20F029
:103EA000D8960101D9A5D8860001D8B66BEF1FF0CE
:103EB0000C0EF76EF60EF66ED7EC01F004EEA5F0E0
:103EC000EE5003E0DFEC01F0FBD70D0EDFEC01F06C
:103ED0000A0EDFEC01F00401A4530001D8A47EEF28
:103EE0001FF004EEA5F0EE5003E0DFEC01F0FBD78D
:103EF0000D0EDFEC01F00A0EDFEC01F0010E040103
:103F0000A45D0001D8A492EF1FF004EEA5F0EE50DE
:103F100003E0DFEC01F0FBD70D0EDFEC01F00A0E41
:103F2000DFEC01F06CEC20F0EDEF1FF0020E010170
:103F30006A5D0001D8A4EDEF1FF00501ED51320DCF
:103F4000F3CF1CF0F4CF1DF026EC02F0000123ECBF
:103F500020F0D8960101D9A5D8860001D8B6C4EFC3
:103F60001FF00C0EF76EFE0EF66ED7EC01F004EEAD
:103F7000A5F0EE5003E0DFEC01F0FBD70D0EDFEC17
:103F800001F00A0EDFEC01F00401A4530001D8A4F3
:103F9000D7EF1FF004EEA5F0EE5003E0DFEC01F0E8
:103FA000FBD70D0EDFEC01F00A0EDFEC01F0010E85
:103FB0000401A45D0001D8A4EBEF1FF004EEA5F00E
:103FC000EE5003E0DFEC01F0FBD70D0EDFEC01F06B
:103FD0000A0EDFEC01F06CEC20F0120023EC20F074
:103FE000D8960101D9A5D8860001D8B60BEF20F0EC
:103FF0000D0EF76E060EF66ED7EC01F003EE0DF027
:10400000EE5003E0DFEC01F0FBD70D0EDFEC01F02A
:104010000A0EDFEC01F0D896060111B7D886000130
:10402000D8B620EF20F003EE0DF0EE5003E0DFEC09
:1040300001F0FBD70D0EDFEC01F00A0EDFEC01F012
:104040006CEC20F012000101D76B000101EEA0F032
:10405000020E016EE86A82B6010ECCEC00F0EF6A47
:1040600001EEA0F084EC00F00101D46F010ED45DEC
:104070000001D8A43EEF20F052EF20F00101D72B31
:104080000501ED510A0DF3CF1CF0F4CF1DF026EC25
:1040900002F0330E0101D75D0001D8A051EF20F0EE
:1040A0001200D3D794908280050E24EC02F0D896AB
:1040B0000101D9A5D8860001D8B66BEF20F00D0E0E
:1040C000F76E0E0EF66ED7EC01F00D0EDFEC01F080
:1040D0000A0EDFEC01F0120094908290D896010154
:1040E000D9A5D8860001D8B682EF20F00D0EF76E64
:1040F000360EF66ED7EC01F00D0EDFEC01F00A0E75
:10410000DFEC01F01200D8960101D9ABD88600018E
:10411000D8B699EF20F002EE76F011EEE2F0030E41
:10412000F36E000E0401185DE1EC02F0EF6A01018C
:10413000D99B0001D8960101D9A5D8860001D8B62F
:10414000AEEF20F00D0EF76E480EF66ED7EC01F0D4
:104150000D0EDFEC01F00A0EDFEC01F001EEE2F0F3
:1041600012EE76F0410EE75204E0E6CFEEFFE82EC5
:10417000FAD7EF6A416A01EEE2F0E86AEE5202E035
:10418000E83EFCD70401186F0101CC6B000101016E
:10419000CC510401185D0001D8A052EF21F0D8964F
:1041A0000101D9A5D8860001D8B6E9EF20F00D0E9F
:1041B000F76E6C0EF66ED7EC01F0040E016E040182
:1041C0001851CCEC00F00D0EDFEC01F00A0EDFEC24
:1041D00001F00001D8960101D9A5D8860001D8B612
:1041E0000FEF21F0690EDFEC01F03D0EDFEC01F086
:1041F000DFEC01F0040E016E0101CC51CCEC00F0BB
:104200000D0EF76E7E0EF66ED7EC01F04150CCEC41
:1042100000F00D0EDFEC01F00A0EDFEC01F0000102
:1042200001EEE2F00101CC51E926000EEA22EF5046
:104230000B6E200E0B5C0001D8A425EF21F00101CC
:10424000CC29416E000152EF21F0D8960101D9A589
:10425000D8860001D8B64CEF21F0690EDFEC01F0F2
:104260003D0EDFEC01F0DFEC01F0DFEC01F0040EBD
:10427000016E0101CC51CCEC00F00D0EF76E8C0EEE
:10428000F66ED7EC01F04150CCEC00F00D0EDFECF7
:1042900001F00A0EDFEC01F000010101CC2B00015E
:1042A000D8A474D700EE43F011EEE2F04104E6CF5B
:1042B000EEFFE82EFCD7EF6A00EE43F010EE43F07D
:1042C000F5EC02F000EE58F011EEE2F0415004017E
:1042D000185DEAEC02F0EF6A41520001D8A474EFD5
:1042E00021F000EE58F0EE6A00EE58F010EE58F0B3
:1042F000F5EC02F001EE31F010EE58F0400EE7520E
:1043000004E0E6CFEEFFE82EFAD7EF6AD896010177
:10431000D9A5D8860001D8B69FEF21F00D0EF76E13
:104320009C0EF66ED7EC01F0040E016E4150CCEC01
:1043300000F00D0EDFEC01F00A0EDFEC01F0D89674
:104340000101D9A5D8860001D8B6BAEF21F00D0E2B
:10435000F76EAA0EF66ED7EC01F000EE43F0EE50C9
:1043600003E0DFEC01F0FBD70D0EDFEC01F00A0EED
:10437000DFEC01F0D8960101D9A5D8860001D8B6A6
:10438000D5EF21F00D0EF76EB80EF66ED7EC01F0FA
:1043900000EE58F0EE5003E0DFEC01F0FBD70D0E1D
:1043A000DFEC01F00A0EDFEC01F00D0EF76EC60E29
:1043B000F66E00EE43F001EC03F0D8A4E4EF21F038
:1043C000DBEC3AF05FEF27F00D0EF76ECE0EF66ED7
:1043D00000EE43F001EC03F0D8A4F3EF21F04DEC34
:1043E00042F05FEF27F00D0EF76ED80EF66E00EE7E
:1043F00043F001EC03F0D8A402EF22F073EC42F09A
:104400005FEF27F00D0EF76EE20EF66E00EE43F052
:1044100001EC03F0D8A411EF22F099EC42F05FEF29
:1044200027F00D0EF76EEC0EF66E00EE43F001EC89
:1044300003F0D8A420EF22F0BFEC42F05FEF27F0AA
:104440000D0EF76EF60EF66E00EE43F001EC03F083
:10445000D8A42FEF22F0E5EC42F05FEF27F00E0E2C
:10446000F76E000EF66E00EE43F001EC03F0D8A4F8
:104470003EEF22F00BEC43F05FEF27F00E0EF76EED
:104480000A0EF66E00EE43F001EC03F0D8A44DEFF7
:1044900022F031EC43F05FEF27F00E0EF76E140EB2
:1044A000F66E00EE43F001EC03F0D8A45CEF22F0CE
:1044B00057EC43F05FEF27F00E0EF76E1E0EF66E10
:1044C00000EE43F001EC03F0D8A46BEF22F07DEC9A
:1044D00043F05FEF27F00E0EF76E280EF66E00EE3B
:1044E00043F001EC03F0D8A47AEF22F0A3EC43F000
:1044F0005FEF27F00E0EF76E320EF66E00EE43F011
:1045000001EC03F0D8A489EF22F0C9EC43F05FEF8F
:1045100027F00E0EF76E3A0EF66E00EE43F001EC49
:1045200003F0D8A498EF22F02FEC44F05FEF27F0CF
:104530000E0EF76E420EF66E00EE43F001EC03F045
:10454000D8A4B3EF22F00601118904EEA5F00E0EF7
:10455000F76E4C0EF66ED9EC02F0EF6A0001F9EC42
:104560001EF05FEF27F00E0EF76E620EF66E00EE95
:1045700043F001EC03F0D8A4CEEF22F0060111992C
:1045800004EEA5F00E0EF76E6C0EF66ED9EC02F08E
:10459000EF6A0001F9EC1EF05FEF27F00E0EF76EE8
:1045A000820EF66E00EE43F001EC03F0D8A4E9EFC2
:1045B00022F00601118B04EEA5F00E0EF76E8C0EA4
:1045C000F66ED9EC02F0EF6A0001F9EC1EF05FEF35
:1045D00027F00E0EF76EA20EF66E00EE43F001EC21
:1045E00003F0D8A404EF23F00601119B04EEA5F01C
:1045F0000E0EF76EAE0EF66ED9EC02F0EF6A000109
:10460000F9EC1EF05FEF27F00E0EF76EC60EF66E99
:1046100000EE43F001EC03F0D8A413EF23F095EC87
:1046200044F05FEF27F00E0EF76ECC0EF66E00EE44
:1046300043F001EC03F0D8A422EF23F0CAEC44F0DD
:104640005FEF27F00E0EF76ED20EF66E00EE43F01F
:1046500001EC03F0D8A431EF23F0FFEC44F05FEF5E
:1046600027F00E0EF76ED80EF66E00EE43F001EC5A
:1046700003F0D8A440EF23F034EC45F05FEF27F0CF
:104680000E0EF76EDE0EF66E00EE43F001EC03F058
:10469000D8A44FEF23F069EC45F05FEF27F00E0E42
:1046A000F76EE40EF66E00EE43F001EC03F0D8A4D2
:1046B0005EEF23F09EEC45F05FEF27F00E0EF76EF5
:1046C000E80EF66E00EE43F001EC03F0D8A46DEFB7
:1046D00023F09EEC45F05FEF27F00E0EF76EEC0E28
:1046E000F66E00EE43F001EC03F0D8A47CEF23F06B
:1046F000E4EC45F05FEF27F00E0EF76EF00EF66E6D
:1047000000EE43F001EC03F0D8A48BEF23F070EC43
:1047100046F05FEF27F00E0EF76EF60EF66E00EE27
:1047200043F001EC03F0D8A49AEF23F01FEC2DF036
:104730005FEF27F00E0EF76EFA0EF66E00EE43F006
:1047400001EC03F0D8A4A9EF23F02EEC2DF05FEFDD
:1047500027F00E0EF76EFE0EF66E00EE43F001EC43
:1047600003F0D8A4B8EF23F052EC2DF05FEF27F060
:104770000F0EF76E040EF66E00EE43F001EC03F040
:10478000D8A4C7EF23F07CEC2DF05FEF27F00F0EDD
:10479000F76E080EF66E00EE43F001EC03F0D8A4BD
:1047A000D6EF23F0F2EC3AF05FEF27F00F0EF76E42
:1047B000100EF66E00EE43F001EC03F0D8A4E5EF26
:1047C00023F02AEC3BF05FEF27F00F0EF76E180E88
:1047D000F66E00EE43F001EC03F0D8A4F4EF23F002
:1047E00062EC3BF05FEF27F00F0EF76E200EF66ED7
:1047F00000EE43F001EC03F0D8A403EF24F09AECB0
:104800003BF05FEF27F00F0EF76E280EF66E00EE0E
:1048100043F001EC03F0D8A412EF24F09BEC3BF042
:104820005FEF27F00F0EF76E300EF66E00EE43F0DE
:1048300001EC03F0D8A421EF24F09CEC3BF05FEFF7
:1048400027F00F0EF76E380EF66E00EE43F001EC17
:1048500003F0D8A430EF24F09DEC3BF05FEF27F09D
:104860000F0EF76E400EF66E00EE43F001EC03F013
:10487000D8A43FEF24F05CEC39F05FEF27F00F0E87
:10488000F76E440EF66E00EE43F001EC03F0D8A490
:104890004EEF24F008EC3AF05FEF27F00F0EF76EC2
:1048A0004C0EF66E00EE43F001EC03F0D8A45DEF81
:1048B00024F0D7EC33F05FEF27F00F0EF76E540EB5
:1048C000F66E00EE43F001EC03F0D8A46CEF24F098
:1048D00012EC34F05FEF27F00F0EF76E5C0EF66E01
:1048E00000EE43F001EC03F0D8A47BEF24F04DEC94
:1048F00034F05FEF27F00F0EF76E640EF66E00EEE9
:1049000043F001EC03F0D8A48AEF24F088EC34F0F3
:104910005FEF27F00F0EF76E6C0EF66E00EE43F0B1
:1049200001EC03F0D8A499EF24F0C3EC34F05FEF6E
:1049300027F00F0EF76E740EF66E00EE43F001ECEA
:1049400003F0D8A4A8EF24F0FEEC34F05FEF27F0DA
:104950000F0EF76E7C0EF66E00EE43F001EC03F0E6
:10496000D8A4B7EF24F039EC35F05FEF27F00F0E45
:10497000F76E840EF66E00EE43F001EC03F0D8A45F
:10498000C6EF24F074EC35F05FEF27F00F0EF76EF2
:104990008C0EF66E00EE43F001EC03F0D8A4D5EFD8
:1049A00024F0A2EC33F05FEF27F00F0EF76E940EB9
:1049B000F66E00EE43F001EC03F0D8A4E4EF24F02F
:1049C000AFEC35F05FEF27F00F0EF76E9C0EF66E32
:1049D00000EE43F001EC03F0D8A4F3EF24F004EC74
:1049E00036F05FEF27F00F0EF76EA40EF66E00EEB6
:1049F00043F001EC03F0D8A402EF25F059EC36F0B7
:104A00005FEF27F00F0EF76EAC0EF66E00EE43F080
:104A100001EC03F0D8A411EF25F0AEEC36F05FEF17
:104A200027F00F0EF76EB40EF66E00EE43F001ECB9
:104A300003F0D8A420EF25F0DEEC41F05FEF27F083
:104A40000F0EF76EBC0EF66E00EE43F001EC03F0B5
:104A5000D8A42FEF25F0FCEC41F05FEF27F00F0E0C
:104A6000F76EC60EF66E00EE43F001EC03F0D8A42C
:104A70003EEF25F0A5EC2CF05FEF27F00F0EF76E60
:104A8000CA0EF66E00EE43F001EC03F0D8A44DEF31
:104A900025F09DEC2CF05FEF27F00F0EF76ED00E97
:104AA000F66E00EE43F001EC03F0D8A45CEF25F0C5
:104AB00041EC54F05FEF27F00F0EF76ED60EF66E56
:104AC00000EE43F001EC03F0D8A46BEF25F0D2EC3C
:104AD0004AF05FEF27F00F0EF76EDC0EF66E00EE79
:104AE00043F001EC03F0D8A47AEF25F05EEC47F038
:104AF0005FEF27F00F0EF76EE20EF66E00EE43F05A
:104B000001EC03F0D8A489EF25F0E5EC4EF05FEF5F
:104B100027F00F0EF76EEA0EF66E00EE43F001EC92
:104B200003F0D8A498EF25F01EEC28F05FEF27F0F3
:104B30000F0EF76EF00EF66E00EE43F001EC03F090
:104B4000D8A4A7EF25F03CEC2BF05FEF27F00F0E79
:104B5000F76EF80EF66E00EE43F001EC03F0D8A409
:104B6000C2EF25F00101D98104EEA5F0100EF76E19
:104B7000000EF66ED9EC02F0EF6A0001F9EC1EF0BF
:104B80005FEF27F0100EF76E0E0EF66E00EE43F09C
:104B900001EC03F0D8A4DDEF25F00101D99104EE7A
:104BA000A5F0100EF76E180EF66ED9EC02F0EF6A53
:104BB0000001F9EC1EF05FEF27F0100EF76E280EE3
:104BC000F66E00EE43F001EC03F0D8A4F8EF25F008
:104BD0000101D98304EEA5F0100EF76E320EF66EC9
:104BE000D9EC02F0EF6A0001F9EC1EF05FEF27F05C
:104BF000100EF76E500EF66E00EE43F001EC03F06F
:104C0000D8A413EF26F00101D99304EEA5F0100EFD
:104C1000F76E5C0EF66ED9EC02F0EF6A0001F9EC6B
:104C20001EF05FEF27F0100EF76E7A0EF66E00EEB4
:104C300043F001EC03F0D8A42EEF26F00101D98552
:104C400004EEA5F0100EF76E860EF66ED9EC02F0AB
:104C5000EF6A0001F9EC1EF05FEF27F0100EF76E1F
:104C60009C0EF66E00EE43F001EC03F0D8A449EF81
:104C700026F00101D99504EEA5F0100EF76EA80EEE
:104C8000F66ED9EC02F0EF6A0001F9EC1EF05FEF6E
:104C900027F0100EF76EC00EF66E00EE43F001EC3A
:104CA00003F0D8A458EF26F066EC27F05FEF27F06A
:104CB000100EF76EC60EF66E00EE43F001EC03F038
:104CC000D8A467EF26F099EC27F05FEF27F0100EDD
:104CD000F76ED00EF66E00EE43F001EC03F0D8A4B0
:104CE00076EF26F023EC2CF05FEF27F0100EF76E36
:104CF000DA0EF66E00EE43F001EC03F0D8A485EF77
:104D000026F0CBEC2CF05FEF27F0100EF76EE40EE0
:104D1000F66E00EE43F001EC03F0D8A494EF26F019
:104D2000CBEC2CF05FEF27F0100EF76EE80EF66E6E
:104D300000EE43F001EC03F0D8A4AFEF26F004013D
:104D4000A46B04EEA5F0100EF76EF20EF66ED9EC21
:104D500002F0EF6A0001F9EC1EF05FEF27F0110E90
:104D6000F76E0E0EF66E00EE43F001EC03F0D8A4E1
:104D7000CBEF26F0010E0401A46F04EEA5F0110E96
:104D8000F76E160EF66ED9EC02F0EF6A0001F9EC40
:104D90001EF05FEF27F0110EF76E400EF66E00EE7C
:104DA00043F001EC03F0D8A4DAEF26F035EC1DF067
:104DB0005FEF27F0110EF76E460EF66E00EE43F031
:104DC00001EC03F0D8A4E9EF26F0ADEC2CF05FEF96
:104DD00027F0110EF76E540EF66E00EE43F001EC64
:104DE00003F0D8A4F8EF26F0B0EC46F05FEF27F020
:104DF000110EF76E5A0EF66E00EE43F001EC03F062
:104E0000D8A407EF27F032EF16F05FEF27F0110E6E
:104E1000F76E620EF66E00EE43F001EC03F0D8A4DC
:104E200016EF27F01AEC42F05FEF27F0110EF76E45
:104E30006A0EF66E00EE43F001EC03F0D8A425EF05
:104E400027F02FEC42F05FEF27F0110EF76E720E95
:104E5000F66E00EE43F001EC03F0D8A434EF27F037
:104E6000E0EC32F05FEF27F0110EF76E760EF66E83
:104E700000EE43F001EC03F0D8A443EF27F067EC19
:104E800041F05FEF27F0110EF76E7E0EF66E00EE2A
:104E900043F001EC03F0D8A452EF27F08BEC41F083
:104EA0005FEF27F0110EF76E840EF66E00EE43F002
:104EB00001EC03F0D8A45FEF27F03EEC41F00401D1
:104EC000A36BA26B0001FEEC18F0120002EECBF017
:104ED000110EF76E8A0EF66ED9EC02F011EEDCF0D0
:104EE000040EE75204E0E6CFEEFFE82EFAD7110EEB
:104EF000F76E920EF66ED9EC02F015EEE4F0060EA7
:104F0000E75204E0E6CFEEFFE82EFAD7110EF76E77
:104F10009C0EF66ED9EC02F0020E016E0501ED5109
:104F2000CCEC00F0EF6A000146EC1DF0EEEC1FF057
:104F300012000501ED510A0DF3CF1CF0F4CF1DF066
:104F400026EC02F00001C2DF12000401A4530001AC
:104F5000D8A4DFEF27F002EECBF0110EF76EA80E0B
:104F6000F66ED9EC02F0020E016EE86A82B8010E0C
:104F7000CCEC00F0020E016EE86A82BA010ECCECB5
:104F800000F0020E016EE86A81B0010ECCEC00F078
:104F9000020E016EE86A81B2010ECCEC00F0020E46
:104FA000016EE86A81B4010ECCEC00F0300EEE6EBA
:104FB000EE6EEE6EEF6A46EC1DF0EEEC1FF0010EA9
:104FC0000401A45D0001D8A41AEF28F002EECBF092
:104FD000110EF76EB00EF66ED9EC02F0020E016EF5
:104FE000E86A82B8010ECCEC00F0020E016EE86AAD
:104FF00082BA010ECCEC00F0020E016EE86A81B0BC
:10500000010ECCEC00F0020E016EE86A81B2010ED6
:10501000CCEC00F0020E016EE86A81B4010ECCEC1B
:1050200000F0300EEE6EEE6EEE6EEF6A46EC1DF0A6
:10503000EEEC1FF0140E24EC02F012000401A45355
:105040000001D8A4ACEF29F002EECBF0110EF76E00
:10505000B80EF66ED9EC02F0020E016EE86A82B864
:10506000010ECCEC00F0020E016EE86A82BA010E6D
:10507000CCEC00F0020E016EE86A81B0010ECCECBF
:1050800000F0020E016EE86A81B2010ECCEC00F075
:10509000020E016EE86A81B4010ECCEC00F0300E15
:1050A000EE6EEE6EEE6EEF6A46EC1DF0EEEC1FF06B
:1050B000140E24EC02F002EECBF0110EF76EC00ECF
:1050C000F66ED9EC02F0020E016E3BC52FF03AC528
:1050D0002EF039C52DF038C52CF0030EFEEC00F093
:1050E0002C0EEE6E020E016E3FC52FF03EC52EF067
:1050F0003DC52DF03CC52CF0030EFEEC00F02C0E4F
:10510000EE6E020E016E43C52FF042C52EF041C572
:105110002DF040C52CF0030EFEEC00F02C0EEE6ED0
:10512000020E016E47C52FF046C52EF045C52DF085
:1051300044C52CF0030EFEEC00F0EF6A46EC1DF0C7
:10514000EEEC1FF0140E24EC02F002EECBF0110E88
:10515000F76EC80EF66ED9EC02F0020E016E086A08
:10516000F6C521F0F5C520F0CFEC00F02C0EEE6E68
:10517000020E016E086AF8C521F0F7C520F0CFECE9
:1051800000F02C0EEE6E020E016E086AFAC521F0D8
:10519000F9C520F0CFEC00F02C0EEE6E020E016E81
:1051A000086AFCC521F0FBC520F0CFEC00F02C0E06
:1051B000EE6E020E016E086AFEC521F0FDC520F0FC
:1051C000CFEC00F02C0EEE6E020E016E086A00C6E7
:1051D00021F0FFC520F0CFEC00F02C0EEE6E020E99
:1051E000016E086A02C621F001C620F0CFEC00F083
:1051F0002C0EEE6E020E016E000ECCEC00F02C0EAA
:10520000EE6E020E016EE86A060111B9010ECCECD9
:1052100000F0EF6A000146EC1DF0EEEC1FF0140EFA
:1052200024EC02F002EECBF0110EF76ED00EF66E0B
:10523000D9EC02F0020E016E086A04C621F003C622
:1052400020F0CFEC00F02C0EEE6E020E016E086A1C
:1052500006C621F005C620F0CFEC00F02C0EEE6E55
:10526000020E016E086A08C621F007C620F0CFECD6
:1052700000F02C0EEE6E020E016E086A0AC621F0D6
:1052800009C620F0CFEC00F02C0EEE6E020E016E7F
:10529000086A0CC621F00BC620F0CFEC00F02C0EF3
:1052A000EE6E020E016E086A0EC621F00DC620F0E9
:1052B000CFEC00F02C0EEE6E020E016E086A10C6E6
:1052C00021F00FC620F0CFEC00F02C0EEE6E020E97
:1052D000016E000ECCEC00F02C0EEE6E020E016E94
:1052E000E86A060111BB010ECCEC00F0EF6A000188
:1052F00046EC1DF0EEEC1FF0140E24EC02F002EE72
:10530000CBF0110EF76ED80EF66ED9EC02F0020E4D
:10531000016E0501ED51CCEC00F02C0EEE6E020E8C
:10532000016E086AE1C521F0E0C520F0CFEC00F085
:105330002C0EEE6E020E016E086AE3C521F0E2C586
:1053400020F0CFEC00F0EF6A000146EC1DF0EEEC2F
:105350001FF0140E24EC02F0010E0401A45D000104
:10536000D8A43BEF2BF002EECBF0110EF76EE00E5F
:10537000F66ED9EC02F0020E016EE86A82B8010EF8
:10538000CCEC00F0020E016EE86A82BA010ECCECA1
:1053900000F0020E016EE86A81B0010ECCEC00F064
:1053A000020E016EE86A81B2010ECCEC00F0020E32
:1053B000016EE86A81B4010ECCEC00F0300EEE6EA6
:1053C000EE6EEE6EEF6A46EC1DF0EEEC1FF0140E82
:1053D00024EC02F002EECBF0110EF76EE80EF66E42
:1053E000D9EC02F0020E016E3BC52FF03AC52EF04B
:1053F00039C52DF038C52CF0030EFEEC00F02C0E54
:10540000EE6E020E016E3FC52FF03EC52EF03DC57B
:105410002DF03CC52CF0030EFEEC00F02C0EEE6ED1
:10542000020E016E43C52FF042C52EF041C52DF08E
:1054300040C52CF0030EFEEC00F02C0EEE6E020EBA
:10544000016E47C52FF046C52EF045C52DF044C569
:105450002CF0030EFEEC00F0EF6A46EC1DF0EEECD3
:105460001FF0140E24EC02F002EECBF0110EF76EDA
:10547000F00EF66ED9EC02F0020E016E086AF6C567
:1054800021F0F5C520F0CFEC00F02C0EEE6E020EF0
:10549000016E086AF8C521F0F7C520F0CFEC00F0E6
:1054A0002C0EEE6E020E016E086AFAC521F0F9C5E7
:1054B00020F0CFEC00F02C0EEE6E020E016E086AAA
:1054C000FCC521F0FBC520F0CFEC00F02C0EEE6EF9
:1054D000020E016E086AFEC521F0FDC520F0CFEC7A
:1054E00000F02C0EEE6E020E016E086A00C621F06E
:1054F000FFC520F0CFEC00F02C0EEE6E020E016E18
:10550000086A02C621F001C620F0CFEC00F02C0E94
:10551000EE6E020E016E000ECCEC00F02C0EEE6E64
:10552000020E016EE86A060111B9010ECCEC00F022
:10553000EF6A000146EC1DF0EEEC1FF0140E24ECB7
:1055400002F002EECBF0110EF76EF80EF66ED9EC0B
:1055500002F0020E016E086A04C621F003C620F0B4
:10556000CFEC00F02C0EEE6E020E016E086A06C63D
:1055700021F005C620F0CFEC00F02C0EEE6E020EEE
:10558000016E086A08C621F007C620F0CFEC00F0D3
:105590002C0EEE6E020E016E086A0AC621F009C6D4
:1055A00020F0CFEC00F02C0EEE6E020E016E086AB9
:1055B0000CC621F00BC620F0CFEC00F02C0EEE6EE6
:1055C000020E016E086A0EC621F00DC620F0CFEC67
:1055D00000F02C0EEE6E020E016E086A10C621F06D
:1055E0000FC620F0CFEC00F02C0EEE6E020E016E16
:1055F000000ECCEC00F02C0EEE6E020E016EE86A8E
:10560000060111BB010ECCEC00F0EF6A000146EC84
:105610001DF0EEEC1FF0140E24EC02F002EECBF0C5
:10562000120EF76E000EF66ED9EC02F0020E016E4D
:105630000501ED51CCEC00F02C0EEE6E020E016E69
:10564000086AE1C521F0E0C520F0CFEC00F02C0E97
:10565000EE6E020E016E086AE3C521F0E2C520F08D
:10566000CFEC00F0EF6A000146EC1DF0EEEC1FF00D
:10567000140E24EC02F0120002EECBF0120EF76EC4
:10568000080EF66ED9EC02F0020E016EE86A82B8DE
:10569000010ECCEC00F0020E016EE86A82BA010E37
:1056A000CCEC00F0020E016EE86A81B0010ECCEC89
:1056B00000F0020E016EE86A81B2010ECCEC00F03F
:1056C000020E016EE86A81B4010ECCEC00F0300EDF
:1056D000EE6EEE6EEE6E2C0EEE6E020E016E3BC5A1
:1056E0002FF03AC52EF039C52DF038C52CF0030E39
:1056F000FEEC00F02C0EEE6E020E016E3FC52FF098
:105700003EC52EF03DC52DF03CC52CF0030EFEEC41
:1057100000F02C0EEE6E020E016E43C52FF042C556
:105720002EF041C52DF040C52CF0030EFEEC00F02C
:105730002C0EEE6E020E016E47C52FF046C52EF000
:1057400045C52DF044C52CF0030EFEEC00F02C0EE8
:10575000EE6E020E016EE86A80BA010ECCEC00F02B
:10576000020E016EE86A81B6010ECCEC00F0020E6A
:10577000016EE86A81B8010ECCEC00F0020E016EF9
:10578000E86A82B6010ECCEC00F0EF6A46EC1DF040
:10579000EEEC1FF0140E24EC02F01200120EF76E65
:1057A000100EF66E01EEDCF001EC03F0D8A4F5EF7C
:1057B0002BF0010E0101CC6F0001040E0101CC5D44
:1057C0000001D8B0F3EF2BF094928292FA0E24EC01
:1057D00002F094928282FA0E24EC02F00101CC2BAA
:1057E0000001D8A4E9D722EF2CF0010E0101CC6F03
:1057F0000001030E0101CC5D0001D8B022EF2CF0B6
:1058000094928292010E1D6EF40E25EC02F0949299
:105810008282C80E24EC02F094928292010E1D6ED8
:10582000F40E25EC02F094928282C80E24EC02F071
:10583000010E1D6E900E25EC02F00101CC2B000133
:10584000D8A4D6D7120001EEDCF0460EEE6E410E63
:10585000EE6E490EEE6E4C0EEE6EEF6A120096EC96
:105860002CF001EE31F0120EF76E140EF66ED9EC3C
:1058700002F0020E016E0501ED51CCEC00F0120EAB
:10588000F76E280EF66ED9EC02F0EF6A000135ECE7
:105890001DF0010E0101CC6F0001040E0101CC5D71
:1058A0000001D8B079EF2CF094928292820E026EB1
:1058B000040E096E010E046EF40E036E030E216ECB
:1058C000E80E206E33EC00F094928282820E026E1B
:1058D000040E096E010E046EF40E036E010E216EAD
:1058E000900E206E33EC00F00101CC2B0001D8A407
:1058F000D3D705EE93F0460EEE6E410EEE6E490ED6
:10590000EE6E4C0EEE6EEF6A9EEC2DF0949282924B
:10591000010E1D6EF40E25EC02F094928282010EAF
:105920001D6EF40E25EC02F0F1D712008298829AD7
:10593000819081928194120012000501266B010171
:105940006B6B0601119700011200010E0501266F15
:10595000010E01016B6F0001120001EE31F084ECC9
:1059600000F00501F36F21C0F4F504EEA5F0120E6E
:10597000F76E3A0EF66ED9EC02F0020E016E086A6E
:10598000F4C521F0F3C520F0CFEC00F0EF6A000180
:10599000F9EC1EF01200CADF2D0E0101CC6F010ED2
:1059A000D46F0001090E0101D45D0001D8B01DEFD4
:1059B0002DF0949882880101CC5124EC02F0949847
:1059C0008298949A828ACC5124EC02F0949A829A1A
:1059D00093908180CC5124EC02F09390819093922B
:1059E0008182CC5124EC02F0939281929394818431
:1059F000CC5124EC02F09394819493928182CC5107
:105A000024EC02F09392819293908180CC5124EC0B
:105A100002F093908190949A828ACC5124EC02F007
:105A2000949A829A94988288CC5124EC02F09498AB
:105A30008298D42B0001D8A4B4D778DF120005EEE9
:105A400093F011EE31F0360EE75204E0E6CFEEFFB0
:105A5000E82EFAD7EF6A9EEC2DF012009392818225
:105A6000C80E24EC02F005EE93F011EE31F0360E84
:105A7000E75204E0E6CFEEFFE82EFAD7EF6A9EEC9D
:105A80002DF0640E24EC02F09392819204EEA5F0C6
:105A9000120EF76E540EF66ED9EC02F0EF6AF9ECC6
:105AA0001EF01200120EF76E5C0EF66E01EE31F073
:105AB00001EC03F0D8A46DEF2DF005012B8504EE69
:105AC000A5F0120EF76E600EF66ED9EC02F0EF6ADA
:105AD0000001F9EC1EF07BEF2DF005012B9504EE93
:105AE000A5F0120EF76E6E0EF66ED9EC02F0EF6AAC
:105AF0000001F9EC1EF0120001EE31F084EC00F030
:105B00000501916F040E196EB00E186E1D6A91C5D5
:105B10001CF09CEC02F08F6F19C090F504EEA5F01C
:105B2000120EF76E7E0EF66ED9EC02F0020E016ECA
:105B30009151CCEC00F0EF6A0001120004EEA5F0E8
:105B4000120EF76E900EF66ED9EC02F015EE93F091
:105B5000320EE75204E0E6CFEEFFE82EFAD7EF6A06
:105B6000F9EC1EF0040E196EB00E186E1D6A91C588
:105B70001CF09CEC02F005018F6F19C090F5949217
:105B8000828205EE93F0E86AEE5202E0E83EFCD72E
:105B9000926F010E0101CC6F00010101CC51050192
:105BA000925D0001D8A098EF30F005EEC6F015EE3A
:105BB00093F0CCC1F3FF010EE1EC02F0EF6A410E6D
:105BC0000501C65D0001D8A4EFEF2DF005EECBF086
:105BD0002E0EEE6E2D0EEE6EEF6A90EF30F0420E4E
:105BE0000501C65D0001D8A401EF2EF005EECBF053
:105BF0002D0EEE6E2E0EEE6EEE6EEE6EEF6A90EFE6
:105C000030F0430E0501C65D0001D8A415EF2EF05B
:105C100005EECBF02D0EEE6E2E0EEE6E2D0EEE6E10
:105C20002E0EEE6EEF6A90EF30F0440E0501C65D69
:105C30000001D8A426EF2EF005EECBF02D0EEE6E6F
:105C40002E0EEE6EEE6EEF6A90EF30F0450E05010F
:105C5000C65D0001D8A434EF2EF005EECBF02E0E79
:105C6000EE6EEF6A90EF30F0460E0501C65D000162
:105C7000D8A447EF2EF005EECBF02E0EEE6EEE6EB2
:105C80002D0EEE6E2E0EEE6EEF6A90EF30F0470E98
:105C90000501C65D0001D8A458EF2EF005EECBF04B
:105CA0002D0EEE6EEE6E2E0EEE6EEF6A90EF30F071
:105CB000480E0501C65D0001D8A469EF2EF005EE7F
:105CC000CBF02E0EEE6EEE6EEE6EEE6EEF6A90EF95
:105CD00030F0490E0501C65D0001D8A478EF2EF022
:105CE00005EECBF02E0EEE6EEE6EEF6A90EF30F01A
:105CF0004A0E0501C65D0001D8A48AEF2EF005EE1C
:105D0000CBF02E0EEE6E2D0EEE6EEE6EEE6EEF6A98
:105D100090EF30F04B0E0501C65D0001D8A49CEF5A
:105D20002EF005EECBF02D0EEE6E2E0EEE6E2D0E3D
:105D3000EE6EEF6A90EF30F04C0E0501C65D00018B
:105D4000D8A4AFEF2EF005EECBF02E0EEE6E2D0E9A
:105D5000EE6E2E0EEE6EEE6EEF6A90EF30F04D0EA0
:105D60000501C65D0001D8A4BEEF2EF005EECBF014
:105D70002D0EEE6EEE6EEF6A90EF30F04E0E0501D6
:105D8000C65D0001D8A4CEEF2EF005EECBF02D0EAF
:105D9000EE6E2E0EEE6EEF6A90EF30F04F0E0501B4
:105DA000C65D0001D8A4DEEF2EF005EECBF02D0E7F
:105DB000EE6EEE6EEE6EEF6A90EF30F0500E050173
:105DC000C65D0001D8A4F1EF2EF005EECBF02E0E4B
:105DD000EE6E2D0EEE6EEE6E2E0EEE6EEF6A90EF04
:105DE00030F0510E0501C65D0001D8A404EF2FF07C
:105DF00005EECBF02D0EEE6EEE6E2E0EEE6E2D0E2F
:105E0000EE6EEF6A90EF30F0520E0501C65D0001B4
:105E1000D8A416EF2FF005EECBF02E0EEE6E2D0E61
:105E2000EE6E2E0EEE6EEF6A90EF30F0530E05011F
:105E3000C65D0001D8A426EF2FF005EECBF02E0EA4
:105E4000EE6EEE6EEE6EEF6A90EF30F0540E0501DE
:105E5000C65D0001D8A434EF2FF005EECBF02D0E77
:105E6000EE6EEF6A90EF30F0550E0501C65D000151
:105E7000D8A445EF2FF005EECBF02E0EEE6EEE6EB1
:105E80002D0EEE6EEF6A90EF30F0560E0501C65DF6
:105E90000001D8A457EF2FF005EECBF02E0EEE6EDA
:105EA000EE6EEE6E2D0EEE6EEF6A90EF30F0570E46
:105EB0000501C65D0001D8A468EF2FF005EECBF018
:105EC0002E0EEE6E2D0EEE6EEE6EEF6A90EF30F04F
:105ED000580E0501C65D0001D8A47BEF2FF005EE3A
:105EE000CBF02D0EEE6E2E0EEE6EEE6E2D0EEE6ED5
:105EF000EF6A90EF30F0590E0501C65D0001D8A49D
:105F00008EEF2FF005EECBF02D0EEE6E2E0EEE6E18
:105F10002D0EEE6EEE6EEF6A90EF30F05A0E050128
:105F2000C65D0001D8A4A0EF2FF005EECBF02D0E3A
:105F3000EE6EEE6E2E0EEE6EEE6EEF6A90EF30F0BD
:105F4000300E0501C65D0001D8A4B2EF2FF005EEBA
:105F5000CBF02D0EEE6EEE6EEE6EEE6EEE6EEF6A26
:105F600090EF30F0310E0501C65D0001D8A4C5EFF9
:105F70002FF005EECBF02E0EEE6E2D0EEE6EEE6EC9
:105F8000EE6EEE6EEF6A90EF30F0320E0501C65DF8
:105F90000001D8A4D8EF2FF005EECBF02E0EEE6E58
:105FA000EE6E2D0EEE6EEE6EEE6EEF6A90EF30F04E
:105FB000330E0501C65D0001D8A4EBEF2FF005EE0E
:105FC000CBF02E0EEE6EEE6EEE6E2D0EEE6EEE6ED3
:105FD000EF6A90EF30F0340E0501C65D0001D8A4E1
:105FE000FDEF2FF005EECBF02E0EEE6EEE6EEE6EA8
:105FF0002D0EEE6EEF6A90EF30F0350E0501C65DA6
:106000000001D8A40FEF30F005EECBF02E0EEE6EAF
:10601000EE6EEE6EEE6EEE6EEF6A90EF30F0360ED4
:106020000501C65D0001D8A422EF30F005EECBF0EB
:106030002D0EEE6E2E0EEE6EEE6EEE6EEE6EEF6AC4
:1060400090EF30F0370E0501C65D0001D8A435EFA2
:1060500030F005EECBF02D0EEE6EEE6E2E0EEE6EE7
:10606000EE6EEE6EEF6A90EF30F0380E0501C65D11
:106070000001D8A448EF30F005EECBF02D0EEE6E07
:10608000EE6EEE6E2E0EEE6EEE6EEF6A90EF30F06C
:10609000390E0501C65D0001D8A45BEF30F005EEB6
:1060A000CBF02D0EEE6EEE6EEE6EEE6E2E0EEE6EF2
:1060B000EF6A90EF30F02F0E0501C65D0001D8A405
:1060C00070EF30F005EECBF02D0EEE6E2E0EEE6E74
:1060D000EE6E2D0EEE6E2E0EEE6EEF6A90EF30F03D
:1060E0003D0E0501C65D0001D8A484EF30F005EE39
:1060F000CBF02D0EEE6E2E0EEE6EEE6EEE6E2D0EC3
:10610000EE6EEF6A90EF30F0200E0501C65D0001E3
:10611000D8A490EF30F005EECBF0200EEE6EEF6AD3
:1061200099EC30F00101CC2B0001D8A4CCEF2DF07C
:10613000120005EECBF0E86AEE5202E0E83EFCD732
:106140000101D46F010ED76F00010101D751D45D59
:106150000001D8A032EF31F005EEC8F015EECBF01B
:10616000D7C1F3FF010EE1EC02F0EF6A2E0E05013C
:10617000C85D0001D8A4E1EF30F0D89605012BA549
:10618000D8860001D8B6C7EF30F093948184820E90
:10619000026E040E096E90C504F08FC503F08EC523
:1061A00021F08DC520F033EC00F0D89605012BA529
:1061B000D8860001D8B6DFEF30F09394819427EFB2
:1061C00031F02D0E0501C85D0001D8A412EF31F0A9
:1061D000D89605012BA5D8860001D8B6F2EF30F08D
:1061E00093948184820E026E040E096E0501905113
:1061F000030DF3CF04F08F51030DF3CF03F0F450F0
:1062000004268EC521F08DC520F033EC00F0D89621
:106210002BA5D8860001D8B610EF31F09394819465
:1062200027EF31F0200E0501C85D0001D8A426EF4C
:1062300031F005019051030DF3CF1DF08F51030D87
:10624000F3CF1CF0F4501D2626EC02F0000190C59F
:106250001DF005018F5125EC02F00101D72B000143
:10626000D8A472D705019051030DF3CF1DF08F51C3
:10627000030DF3CF1CF0F4501D2626EC02F00001B4
:106280001200000E0DEC02F00501306F2DC031F54B
:10629000176A166A156A8F0E146E31C511F030C573
:1062A00010F0D0EC04F018EC04F013C0D2F112C0DE
:1062B000D1F111C0D0F110C0CFF1136A126A200ED3
:1062C000116E810E106ED2C117F0D1C116F0D0C17F
:1062D00015F0CFC114F080EC04F013C02FF012C001
:1062E0002EF011C02DF010C02CF02FC013F02EC0D6
:1062F00012F02DC011F02CC010F02FC517F02EC5D4
:1063000016F02DC515F02CC514F080EC04F013C068
:106310003BF512C03AF511C039F510C038F53BC550
:1063200013F03AC512F039C511F038C510F04BC55D
:1063300017F04AC516F049C515F048C514F07EECB3
:1063400003F013C03BF512C03AF511C039F510C087
:1063500038F5010E0DEC02F0326F2DC033F5176ADF
:10636000166A156A8F0E146E33C511F032C510F01F
:10637000D0EC04F018EC04F013C0D2F112C0D1F14B
:1063800011C0D0F110C0CFF1136A126A200E116E45
:10639000810E106ED2C117F0D1C116F0D0C115F028
:1063A000CFC114F080EC04F013C02FF012C02EF017
:1063B00011C02DF010C02CF02FC013F02EC012F021
:1063C0002DC011F02CC010F02FC517F02EC516F0FF
:1063D0002DC515F02CC514F080EC04F013C03FF56A
:1063E00012C03EF511C03DF510C03CF53FC513F09D
:1063F0003EC512F03DC511F03CC510F04FC517F079
:106400004EC516F04DC515F04CC514F07EEC03F0EA
:1064100013C03FF512C03EF511C03DF510C03CF56C
:10642000020E0DEC02F0346F2DC035F5176A166AB6
:10643000156A8F0E146E35C511F034C510F0D0EC0E
:1064400004F018EC04F013C0D2F112C0D1F111C065
:10645000D0F110C0CFF1136A126A200E116E810EB6
:10646000106ED2C117F0D1C116F0D0C115F0CFC156
:1064700014F080EC04F013C02FF012C02EF011C005
:106480002DF010C02CF02FC013F02EC012F02DC034
:1064900011F02CC010F02FC517F02EC516F02DC529
:1064A00015F02CC514F080EC04F013C043F512C0B5
:1064B00042F511C041F510C040F543C513F042C587
:1064C00012F041C511F040C510F053C517F052C588
:1064D00016F051C515F050C514F07EEC03F013C052
:1064E00043F512C042F511C041F510C040F5030E4E
:1064F0000DEC02F0366F2DC037F5176A166A156A73
:106500008F0E146E37C511F036C510F0D0EC04F0C4
:1065100018EC04F013C0D2F112C0D1F111C0D0F1C7
:1065200010C0CFF1136A126A200E116E810E106E28
:10653000D2C117F0D1C116F0D0C115F0CFC114F0FF
:1065400080EC04F013C02FF012C02EF011C02DF01B
:1065500010C02CF02FC013F02EC012F02DC011F07F
:106560002CC010F02FC517F02EC516F02DC515F054
:106570002CC514F080EC04F013C047F512C046F5AA
:1065800011C045F510C044F547C513F046C512F0DB
:1065900045C511F044C510F057C517F056C516F0A3
:1065A00055C515F054C514F07EEC03F013C047F543
:1065B00012C046F511C045F510C044F500011200A7
:1065C00004EEA5F0120EF76E9A0EF66ED9EC02F0FC
:1065D000EF6AF9EC1EF00A0E24EC02F052DE04EE33
:1065E000A5F0120EF76EC00EF66ED9EC02F0020E98
:1065F000016E3BC52FF03AC52EF039C52DF038C5D8
:106600002CF0030EFEEC00F0120EF76ED00EF66EBC
:10661000D9EC02F0020E016E086A31C521F030C5D6
:1066200020F0CFEC00F0290EEE6EEF6AF9EC1EF0D0
:1066300004EEA5F0120EF76EDA0EF66ED9EC02F04B
:10664000020E016E3FC52FF03EC52EF03DC52DF068
:106650003CC52CF0030EFEEC00F0120EF76EEA0EB5
:10666000F66ED9EC02F0020E016E086A33C521F015
:1066700032C520F0CFEC00F0290EEE6EEF6AF9EC97
:106680001EF004EEA5F0120EF76EF40EF66ED9ECC5
:1066900002F0020E016E43C52FF042C52EF041C537
:1066A0002DF040C52CF0030EFEEC00F0130EF76E3B
:1066B000040EF66ED9EC02F0020E016E086A35C5C2
:1066C00021F034C520F0CFEC00F0290EEE6EEF6A19
:1066D000F9EC1EF004EEA5F0130EF76E0E0EF66E3A
:1066E000D9EC02F0020E016E47C52FF046C52EF020
:1066F00045C52DF044C52CF0030EFEEC00F0130E42
:10670000F76E1E0EF66ED9EC02F0020E016E086AEC
:1067100037C521F036C520F0CFEC00F0290EEE6E23
:10672000EF6AF9EC1EF004EEA5F0130EF76E280EDA
:10673000F66ED9EC02F0EF6AF9EC1EF00A0E24ECCA
:1067400002F01200130EF76E4E0EF66E01EE31F0EF
:1067500001EC03F0D8A4BCEF33F0010E01016C6F23
:1067600004EEA5F0130EF76E520EF66ED9EC02F0A1
:10677000EF6A0001F9EC1EF0130EF76E6E0EF66E66
:1067800001EE31F001EC03F0D8A4D5EF33F00101B4
:106790006C6B04EEA5F0130EF76E720EF66ED9EC6C
:1067A00002F0EF6A0001F9EC1EF01200120001EE97
:1067B00031F084EC00F020C010F021C011F022C0B4
:1067C00012F023C013F0D2EC04F013C05BF512C03A
:1067D0005AF511C059F510C058F501EEA0F0020E9F
:1067E000016E5BC52FF05AC52EF059C52DF058C566
:1067F0002CF0030EFEEC00F0EF6A04EEA5F0130E91
:10680000F76E8E0EF66ED9EC02F011EEA0F0140EBB
:10681000E75204E0E6CFEEFFE82EFAD7EF6AF9EC94
:106820001EF0120001EE31F084EC00F020C010F0F8
:1068300021C011F022C012F023C013F0D2EC04F0FA
:1068400013C05FF512C05EF511C05DF510C05CF5B8
:1068500001EEA0F0020E016E5FC52FF05EC52EF0B6
:106860005DC52DF05CC52CF0030EFEEC00F0EF6A68
:1068700004EEA5F0130EF76EA40EF66ED9EC02F03E
:1068800011EEA0F0140EE75204E0E6CFEEFFE82E82
:10689000FAD7EF6AF9EC1EF0120001EE31F084EC49
:1068A00000F020C010F021C011F022C012F023C06F
:1068B00013F0D2EC04F013C063F512C062F511C0FE
:1068C00061F510C060F501EEA0F0020E016E63C527
:1068D0002FF062C52EF061C52DF060C52CF0030EBF
:1068E000FEEC00F0EF6A04EEA5F0130EF76EBA0EA0
:1068F000F66ED9EC02F011EEA0F0140EE75204E0AF
:10690000E6CFEEFFE82EFAD7EF6AF9EC1EF01200A0
:1069100001EE31F084EC00F020C010F021C011F045
:1069200022C012F023C013F0D2EC04F013C067F5BC
:1069300012C066F511C065F510C064F501EEA0F057
:10694000020E016E67C52FF066C52EF065C52DF0ED
:1069500064C52CF0030EFEEC00F0EF6A04EEA5F027
:10696000130EF76ED00EF66ED9EC02F011EEA0F019
:10697000140EE75204E0E6CFEEFFE82EFAD7EF6AF6
:10698000F9EC1EF0120001EE31F084EC00F020C0B2
:1069900010F021C011F022C012F023C013F0D2EC8D
:1069A00004F013C06BF512C06AF511C069F510C090
:1069B00068F501EEA0F0020E016E6BC52FF06AC5FE
:1069C0002EF069C52DF068C52CF0030EFEEC00F02A
:1069D000EF6A04EEA5F0130EF76EE60EF66ED9EC34
:1069E00002F011EEA0F0140EE75204E0E6CFEEFF45
:1069F000E82EFAD7EF6AF9EC1EF0120001EE31F042
:106A000084EC00F020C010F021C011F022C012F080
:106A100023C013F0D2EC04F013C06FF512C06EF572
:106A200011C06DF510C06CF501EEA0F0020E016E04
:106A30006FC52FF06EC52EF06DC52DF06CC52CF016
:106A4000030EFEEC00F0EF6A04EEA5F0130EF76EF5
:106A5000FC0EF66ED9EC02F011EEA0F0140EE75227
:106A600004E0E6CFEEFFE82EFAD7EF6AF9EC1EF06D
:106A7000120001EE31F084EC00F020C010F021C0D3
:106A800011F022C012F023C013F0D2EC04F013C0B6
:106A900073F512C072F511C071F510C070F501EEFA
:106AA000A0F0020E016E73C52FF072C52EF071C5F5
:106AB0002DF070C52CF0030EFEEC00F0EF6A04EE32
:106AC000A5F0140EF76E120EF66ED9EC02F011EE70
:106AD000A0F0140EE75204E0E6CFEEFFE82EFAD75E
:106AE000EF6AF9EC1EF0120001EE31F084EC00F0D8
:106AF00020C010F021C011F022C012F023C013F00A
:106B0000D2EC04F013C077F512C076F511C075F51C
:106B100010C074F501EEA0F0020E016E77C52FF0E3
:106B200076C52EF075C52DF074C52CF0030EFEEC65
:106B300000F0EF6A04EEA5F0140EF76E280EF66E64
:106B4000D9EC02F011EEA0F0140EE75204E0E6CF0B
:106B5000EEFFE82EFAD7EF6AF9EC1EF0120001EE14
:106B600031F084EC00F020C010F021C011F022C000
:106B700012F023C013F0D2EC04F013C0D2F112C013
:106B8000D1F111C0D0F110C0CFF16F0E136E120E03
:106B9000126E030E116E750E106ED2C117F0D1C1B8
:106BA00016F0D0C115F0CFC114F080EC04F013C082
:106BB0004BF512C04AF511C049F510C048F501EE79
:106BC000A0F0020E016E4BC52FF04AC52EF049C54C
:106BD0002DF048C52CF0030EFEEC00F0EF6A04EE39
:106BE000A5F0140EF76E3E0EF66ED9EC02F011EE23
:106BF000A0F0140EE75204E0E6CFEEFFE82EFAD73D
:106C0000EF6AF9EC1EF0120001EE31F084EC00F0B6
:106C100020C010F021C011F022C012F023C013F0E8
:106C2000D2EC04F013C0D2F112C0D1F111C0D0F1F6
:106C300010C0CFF16F0E136E120E126E030E116E96
:106C4000750E106ED2C117F0D1C116F0D0C115F07B
:106C5000CFC114F080EC04F013C04FF512C04EF514
:106C600011C04DF510C04CF501EEA0F0020E016E02
:106C70004FC52FF04EC52EF04DC52DF04CC52CF054
:106C8000030EFEEC00F0EF6A04EEA5F0140EF76EB2
:106C9000640EF66ED9EC02F011EEA0F0140EE7527D
:106CA00004E0E6CFEEFFE82EFAD7EF6AF9EC1EF02B
:106CB000120001EE31F084EC00F020C010F021C091
:106CC00011F022C012F023C013F0D2EC04F013C074
:106CD000D2F112C0D1F111C0D0F110C0CFF16F0EBE
:106CE000136E120E126E030E116E750E106ED2C15F
:106CF00017F0D1C116F0D0C115F0CFC114F080EC5F
:106D000004F013C053F512C052F511C051F510C074
:106D100050F501EEA0F0020E016E53C52FF052C5E2
:106D20002EF051C52DF050C52CF0030EFEEC00F0F6
:106D3000EF6A04EEA5F0140EF76E8A0EF66ED9EC2B
:106D400002F011EEA0F0140EE75204E0E6CFEEFFE1
:106D5000E82EFAD7EF6AF9EC1EF0120001EE31F0DE
:106D600084EC00F020C010F021C011F022C012F01D
:106D700023C013F0D2EC04F013C0D2F112C0D1F151
:106D800011C0D0F110C0CFF16F0E136E120E126E43
:106D9000030E116E750E106ED2C117F0D1C116F030
:106DA000D0C115F0CFC114F080EC04F013C057F53A
:106DB00012C056F511C055F510C054F501EEA0F003
:106DC000020E016E57C52FF056C52EF055C52DF099
:106DD00054C52CF0030EFEEC00F0EF6A04EEA5F0B3
:106DE000140EF76EB00EF66ED9EC02F011EEA0F0B4
:106DF000140EE75204E0E6CFEEFFE82EFAD7EF6A72
:106E0000F9EC1EF012003BC513F03AC512F039C57B
:106E100011F038C510F05BC517F05AC516F059C50A
:106E200015F058C514F00AEC03F00108D8B433EF9C
:106E300037F0C4EC37F06BC513F06AC512F069C5C2
:106E400011F068C510F03BC517F03AC516F039C50A
:106E500015F038C514F00AEC03F00108D8B433EF8C
:106E600037F090EC38F03FC513F03EC512F03DC549
:106E700011F03CC510F05FC517F05EC516F05DC59A
:106E800015F05CC514F00AEC03F00108D8B463EF08
:106E900037F0F7EC37F06FC513F06EC512F06DC523
:106EA00011F06CC510F03FC517F03EC516F03DC59A
:106EB00015F03CC514F00AEC03F00108D8B463EFF8
:106EC00037F0C3EC38F043C513F042C512F041C5AA
:106ED00011F040C510F063C517F062C516F061C52A
:106EE00015F060C514F00AEC03F00108D8B493EF74
:106EF00037F02AEC38F073C513F072C512F071C583
:106F000011F070C510F043C517F042C516F041C529
:106F100015F040C514F00AEC03F00108D8B493EF63
:106F200037F0F6EC38F047C513F046C512F045C50A
:106F300011F044C510F067C517F066C516F065C5B9
:106F400015F064C514F00AEC03F00108D8B4C3EFDF
:106F500037F05DEC38F077C513F076C512F075C5E3
:106F600011F074C510F047C517F046C516F045C5B9
:106F700015F044C514F00AEC03F00108D8B4C3EFCF
:106F800037F029EC39F0120004EEA5F0140EF76E7C
:106F9000D60EF66ED9EC02F0020E016E5BC52FF034
:106FA0005AC52EF059C52DF058C52CF0030EFEEC35
:106FB00000F0150EF76E020EF66ED9EC02F0020E1E
:106FC000016E3BC52FF03AC52EF039C52DF038C5FE
:106FD0002CF0030EFEEC00F0760EEE6E2E0EEE6E32
:106FE000EF6AF9EC1EF0640E24EC02F0120004EEDD
:106FF000A5F0150EF76E100EF66ED9EC02F0020E2B
:10700000016E5FC52FF05EC52EF05DC52DF05CC52D
:107010002CF0030EFEEC00F0150EF76E3C0EF66E33
:10702000D9EC02F0020E016E3FC52FF03EC52EF0E6
:107030003DC52DF03CC52CF0030EFEEC00F0760EA5
:10704000EE6E2E0EEE6EEF6AF9EC1EF0640E24EC7E
:1070500002F0120004EEA5F0150EF76E4A0EF66E61
:10706000D9EC02F0020E016E63C52FF062C52EF05E
:1070700061C52DF060C52CF0030EFEEC00F0150E7E
:10708000F76E760EF66ED9EC02F0020E016E43C575
:107090002FF042C52EF041C52DF040C52CF0030E57
:1070A000FEEC00F0760EEE6E2E0EEE6EEF6AF9EC50
:1070B0001EF0640E24EC02F0120004EEA5F0150E92
:1070C000F76E840EF66ED9EC02F0020E016E67C503
:1070D0002FF066C52EF065C52DF064C52CF0030EAB
:1070E000FEEC00F0150EF76EB00EF66ED9EC02F065
:1070F000020E016E47C52FF046C52EF045C52DF096
:1071000044C52CF0030EFEEC00F0760EEE6E2E0E53
:10711000EE6EEF6AF9EC1EF0640E24EC02F0120041
:1071200004EEA5F0150EF76EBE0EF66ED9EC02F069
:10713000020E016E6BC52FF06AC52EF069C52DF0E9
:1071400068C52CF0030EFEEC00F0150EF76EEA0E8B
:10715000F66ED9EC02F0020E016E3BC52FF03AC577
:107160002EF039C52DF038C52CF0030EFEEC00F0E2
:10717000760EEE6E2E0EEE6EEF6AF9EC1EF0640ED9
:1071800024EC02F0120004EEA5F0150EF76EF80ED6
:10719000F66ED9EC02F0020E016E6FC52FF06EC5CF
:1071A0002EF06DC52DF06CC52CF0030EFEEC00F03A
:1071B000160EF76E240EF66ED9EC02F0020E016E7A
:1071C0003FC52FF03EC52EF03DC52DF03CC52CF03F
:1071D000030EFEEC00F0760EEE6E2E0EEE6EEF6AF3
:1071E000F9EC1EF0640E24EC02F0120004EEA5F09F
:1071F000160EF76E320EF66ED9EC02F0020E016E2C
:1072000073C52FF072C52EF071C52DF070C52CF02E
:10721000030EFEEC00F0160EF76E5E0EF66ED9EC65
:1072200002F0020E016E43C52FF042C52EF041C59B
:107230002DF040C52CF0030EFEEC00F0760EEE6E45
:107240002E0EEE6EEF6AF9EC1EF0640E24EC02F0E6
:10725000120004EEA5F0160EF76E6C0EF66ED9EC69
:1072600002F0020E016E77C52FF076C52EF075C5BF
:107270002DF074C52CF0030EFEEC00F0160EF76E28
:10728000980EF66ED9EC02F0020E016E47C52FF093
:1072900046C52EF045C52DF044C52CF0030EFEEC7E
:1072A00000F0760EEE6E2E0EEE6EEF6AF9EC1EF02A
:1072B000640E24EC02F01200160EF76EA60EF66EA7
:1072C00001EE31F001EC03F0D8A475EF39F00501BF
:1072D000786B04EEA5F0160EF76EAA0EF66ED9ECDA
:1072E00002F0EF6A0001F9EC1EF0160EF76ECA0EFE
:1072F000F66E01EE31F001EC03F0D8A48FEF39F017
:10730000010E0501786F04EEA5F0160EF76ECE0E95
:10731000F66ED9EC02F0EF6A0001F9EC1EF0160EE1
:10732000F76EF20EF66E01EE31F001EC03F0D8A428
:10733000A9EF39F0020E0501786F04EEA5F0160EE4
:10734000F76EFA0EF66ED9EC02F0EF6A0001F9EC76
:107350001EF01200010E0501785D0001D8A4CFEFE8
:1073600039F03BC513F03AC512F039C511F038C5F4
:1073700010F03FC517F03EC516F03DC515F03CC5F1
:1073800014F042EC03F00108D8B4CCEF39F0060158
:1073900011830001CEEF39F0060111930001020EB6
:1073A0000501785D0001D8A407EF3AF03FC513F05E
:1073B0003EC512F03DC511F03CC510F07CC517F07C
:1073C0007BC516F07AC515F079C514F00AEC03F008
:1073D000356E3FC513F03EC512F03DC511F03CC5FA
:1073E00010F03BC517F03AC516F039C515F038C591
:1073F00014F00AEC03F03510D8B404EF3AF00601AB
:107400001183000106EF3AF006011193000112000A
:1074100001EE31F084EC00F020C010F021C011F03A
:1074200022C012F023C013F0D2EC04F013C07CF59C
:1074300012C07BF511C07AF510C079F51200120068
:1074400001011B6B00019EAA28EF3AF0AECF1BF1A1
:1074500012009EB82DEF3AF0FCD71BC1ADFF120011
:10746000010E0501D85D0001D8A441EF3AF08288F1
:10747000FA0E24EC02F08298010E1D6E2C0E25EC03
:1074800002F0020E0501D85D0001D8A449EF3AF0E0
:107490008288030E0501D85D0001D8A451EF3AF0AF
:1074A0008298040E0501D85D0001D8A45AEF3AF085
:1074B0003CEC2BF0050E0501D85D0001D8A468EF67
:1074C0003AF082789498010E1D6E2C0E25EC02F095
:1074D0001200010E0501D95D0001D8A47AEF3AF03F
:1074E000828AFA0E24EC02F0829A010E1D6E2C0E96
:1074F00025EC02F0020E0501D95D0001D8A482EF4F
:107500003AF0828A030E0501D95D0001D8A48AEF02
:107510003AF0829A040E0501D95D0001D8A493EFD8
:107520003AF03CEC2BF0050E0501D95D0001D8A422
:10753000A1EF3AF0827A949A010E1D6E2C0E25EC82
:1075400002F01200010E0501DA5D0001D8A4B3EFCC
:107550003AF08180FA0E24EC02F08190010E1D6E4B
:107560002C0E25EC02F0020E0501DA5D0001D8A414
:10757000BBEF3AF08180030E0501DA5D0001D8A46B
:10758000C3EF3AF08190040E0501DA5D0001D8A442
:10759000CCEF3AF03CEC2BF0050E0501DA5D000172
:1075A000D8A4DAEF3AF081709390010E1D6E2C0E84
:1075B00025EC02F01200310E0101315D0001D8A46A
:1075C000E5EF3AF0010E0101E16F0001320E010119
:1075D000315D0001D8A4F0EF3AF0020E0101E16F35
:1075E00000011200310E0101315D0001D8A4FCEF51
:1075F0003AF0010E0501D86F0001320E0101315D34
:107600000001D8A407EF3BF0020E0501D86F00017E
:10761000330E0101315D0001D8A412EF3BF0030EDF
:107620000501D86F0001340E0101315D0001D8A4BD
:107630001DEF3BF0040E0501D86F0001350E01016E
:10764000315D0001D8A428EF3BF0050E0501D86F8D
:1076500000011200310E0101315D0001D8A434EFA8
:107660003BF0010E0501D96F0001320E0101315DC1
:107670000001D8A43FEF3BF0020E0501D96F0001D5
:10768000330E0101315D0001D8A44AEF3BF0030E37
:107690000501D96F0001340E0101315D0001D8A44C
:1076A00055EF3BF0040E0501D96F0001350E0101C5
:1076B000315D0001D8A460EF3BF0050E0501D96FE4
:1076C00000011200310E0101315D0001D8A46CEF00
:1076D0003BF0010E0501DA6F0001320E0101315D50
:1076E0000001D8A477EF3BF0020E0501DA6F00012C
:1076F000330E0101315D0001D8A482EF3BF0030E8F
:107700000501DA6F0001340E0101315D0001D8A4DA
:107710008DEF3BF0040E0501DA6F0001350E01011B
:10772000315D0001D8A498EF3BF0050E0501DA6F3A
:1077300000011200120012001200120094928282C4
:10774000D8960101D9A1D8860001D8B6B4EF3BF094
:10775000170EF76E2A0EF66ED7EC01F00D0EDFEC69
:1077600001F00A0EDFEC01F0D896060111ABD886C5
:107770000001D8B60EEF3DF081A8C1EF3BF03AEF23
:1077800041F0E86A80BA010E356EE86A81B6010EF2
:107790003510D8B4CEEF3BF0AEEF3FF0D8960501F0
:1077A000EEA9D8860001D8B6F3EF3BF00101CE6B0D
:1077B000010ECD6F00010101CD5106010B5D0101EC
:1077C000CE5106010C590001D8A0F1EF3BF0010E9B
:1077D00024EC02F00101CD2BD8B4CE2B0001D8A4AB
:1077E000E9D793948194060109510501F35D0601DF
:1077F0000A510501F4590001D8B001EF3CF0A5ECA5
:1078000027F081A806EF3CF03AEF41F0E86A80BA31
:10781000010E356EE86A81B6010E3510D8B413EF4B
:107820003CF06CEF3FF0D8960501EEABD886000136
:10783000D8B638EF3CF00101CE6B010ECD6F0001E0
:107840000101CD510601095D0101CE5106010A5920
:107850000001D8A036EF3CF0010E24EC02F001014B
:10786000CD2BD8B4CE2B0001D8A4E9D79392819226
:10787000060107510501F35D060108510501F459A0
:107880000001D8B046EF3CF0A5EC27F081A84BEF03
:107890003CF03AEF41F0E86A80BA010E356EE86AD2
:1078A00081B6010E3510D8B458EF3CF02AEF3FF006
:1078B000D8960501EEADD8860001D8B67DEF3CF034
:1078C0000101CE6B010ECD6F00010101CD5106010A
:1078D000075D0101CE51060108590001D8A07BEFD8
:1078E0003CF0010E24EC02F00101CD2BD8B4CE2BDC
:1078F0000001D8A4E9D793908190060105510501B4
:10790000F35D060106510501F4590001D8B08BEF73
:107910003CF0A5EC27F081A890EF3CF03AEF41F065
:10792000E86A80BA010E356EE86A81B6010E35103C
:10793000D8B49DEF3CF0E8EF3EF0D8960501EEAFED
:10794000D8860001D8B6C2EF3CF00101CE6B010E23
:10795000CD6F00010101CD510601055D0101CE5140
:10796000060106590001D8A0C0EF3CF0010E24EC3E
:1079700002F00101CD2BD8B4CE2B0001D8A4E9D759
:10798000949A829A060103510501F35D06010451A0
:107990000501F4590001D8B0D0EF3CF0A5EC27F078
:1079A00081A8D5EF3CF03AEF41F0E86A80BA010EC9
:1079B000356EE86A81B6010E3510D8B4E2EF3CF0BE
:1079C000A6EF3EF0D896060111A1D8860001D8B6E0
:1079D00007EF3DF00101CE6B010ECD6F00010101FB
:1079E000CD510601035D0101CE510601045900018C
:1079F000D8A005EF3DF0010E24EC02F00101CD2BE3
:107A0000D8B4CE2B0001D8A4E9D79498829881A845
:107A10000CEF3DF03AEF41F05EEF3EF081A813EF3E
:107A20003DF03AEF41F0E86A80BA010E356EE86A3F
:107A300081B6010E3510D8B420EF3DF0F3EF40F0E1
:107A4000D8960501EEA9D8860001D8B645EF3DF0DD
:107A50000101CE6B010ECD6F00010101CD51060178
:107A6000035D0101CE51060104590001D8A043EF86
:107A70003DF0010E24EC02F00101CD2BD8B4CE2B49
:107A80000001D8A4E9D79498829806010551050110
:107A9000F35D060106510501F4590001D8B053EF1A
:107AA0003DF0A5EC27F081A858EF3DF03AEF41F00A
:107AB000E86A80BA010E356EE86A81B6010E3510AB
:107AC000D8B465EF3DF0B1EF40F0D8960501EEABCC
:107AD000D8860001D8B68AEF3DF00101CE6B010EC9
:107AE000CD6F00010101CD510601055D0101CE51AF
:107AF000060106590001D8A088EF3DF0010E24ECE4
:107B000002F00101CD2BD8B4CE2B0001D8A4E9D7C7
:107B1000949A829A060107510501F35D0601085106
:107B20000501F4590001D8B098EF3DF0A5EC27F01D
:107B300081A89DEF3DF03AEF41F0E86A80BA010E6E
:107B4000356EE86A81B6010E3510D8B4AAEF3DF063
:107B50006FEF40F0D8960501EEADD8860001D8B69B
:107B6000CFEF3DF00101CE6B010ECD6F00010101A1
:107B7000CD510601075D0101CE51060108590001F2
:107B8000D8A0CDEF3DF0010E24EC02F00101CD2B89
:107B9000D8B4CE2B0001D8A4E9D7939081900601E8
:107BA00009510501F35D06010A510501F45900016F
:107BB000D8B0DDEF3DF0A5EC27F081A8E2EF3DF075
:107BC0003AEF41F0E86A80BA010E356EE86A81B694
:107BD000010E3510D8B4EFEF3DF02DEF40F0D89600
:107BE0000501EEAFD8860001D8B614EF3EF00101D2
:107BF000CE6B010ECD6F00010101CD510601095D73
:107C00000101CE5106010A590001D8A012EF3EF041
:107C1000010E24EC02F00101CD2BD8B4CE2B0001D3
:107C2000D8A4E9D79392819206010B510501F35D27
:107C300006010C510501F4590001D8B022EF3EF0C5
:107C4000A5EC27F081A827EF3EF03AEF41F0E86A73
:107C500080BA010E356EE86A81B6010E3510D8B4CF
:107C600034EF3EF0EBEF3FF0D896060111A1D88635
:107C70000001D8B659EF3EF00101CE6B010ECD6F79
:107C800000010101CD5106010B5D0101CE5106013C
:107C90000C590001D8A057EF3EF0010E24EC02F081
:107CA0000101CD2BD8B4CE2B0001D8A4E9D79394F1
:107CB000819481A85EEF3EF03AEF41F005012B9DE3
:107CC000D896060111B7D8860001D8B66AEF3EF003
:107CD000A5EC27F0ABEF18F0D896060111A3D886D3
:107CE0000001D8B676EF3EF0ABEF18F094928282A6
:107CF000D8960101D9A1D8860001D8B68CEF3EF004
:107D0000170EF76E420EF66ED7EC01F00D0EDFEC9B
:107D100001F00A0EDFEC01F0D896060111A9D88611
:107D20000001D8B6DAEF3FF081A899EF3EF03AEFC4
:107D300041F0010E80BAE86A356E010E81B6E86A3C
:107D40003514D8B4A6EF3EF03AEF41F0D8960501CD
:107D5000EEA9D8860001D8B6CBEF3EF00101CE6B7C
:107D6000010ECD6F00010101CD510501F55D01014D
:107D7000CE510501F6590001D8A0C9EF3EF0010E21
:107D800024EC02F00101CD2BD8B4CE2B0001D8A4F5
:107D9000E9D7949882880501F751F35DF851F459B9
:107DA0000001D8B0D6EF3EF0A5EC27F081A8DBEFBC
:107DB0003EF03AEF41F0010E80BAE86A356E010EEE
:107DC00081B6E86A3514D8B4E8EF3EF09DEF3CF098
:107DD000D8960501EEABD8860001D8B60DEF3FF07E
:107DE0000101CE6B010ECD6F00010101CD510501E6
:107DF000F75D0101CE510501F8590001D8A00BEF44
:107E00003FF0010E24EC02F00101CD2BD8B4CE2BB3
:107E10000001D8A4E9D7949A828A0501F951F35D4B
:107E2000FA51F4590001D8B018EF3FF0A5EC27F053
:107E300081A81DEF3FF03AEF41F0010E80BAE86AE9
:107E4000356E010E81B6E86A3514D8B42AEF3FF0DA
:107E500058EF3CF0D8960501EEADD8860001D8B6B3
:107E60004FEF3FF00101CE6B010ECD6F000101011C
:107E7000CD510501F95D0101CE510501FA5900010D
:107E8000D8A04DEF3FF0010E24EC02F00101CD2B04
:107E9000D8B4CE2B0001D8A4E9D7939081800501F6
:107EA000FB51F35DFC51F4590001D8B05AEF3FF09B
:107EB000A5EC27F081A85FEF3FF03AEF41F0010E0B
:107EC00080BAE86A356E010E81B6E86A3514D8B416
:107ED0006CEF3FF013EF3CF0D8960501EEAFD8867B
:107EE0000001D8B691EF3FF00101CE6B010ECD6FCE
:107EF00000010101CD510501FB5D0101CE510501DC
:107F0000FC590001D8A08FEF3FF0010E24EC02F0E5
:107F10000101CD2BD8B4CE2B0001D8A4E9D7939280
:107F200081820501FD51F35DFE51F4590001D8B085
:107F30009CEF3FF0A5EC27F081A8A1EF3FF03AEFCE
:107F400041F0010E80BAE86A356E010E81B6E86A2A
:107F50003514D8B4AEEF3FF0CEEF3BF0D896060123
:107F600011A1D8860001D8B6D3EF3FF00101CE6B46
:107F7000010ECD6F00010101CD510501FD5D010133
:107F8000CE510501FE590001D8A0D1EF3FF0010EFE
:107F900024EC02F00101CD2BD8B4CE2B0001D8A4E3
:107FA000E9D79394818481A8D8EF3FF03AEF41F06C
:107FB0001DEF41F081A8DFEF3FF03AEF41F0010EF5
:107FC00080BAE86A356E010E81B6E86A3514D8B415
:107FD000EBEF3FF049D6D8960501EEA9D88600010F
:107FE000D8B610EF40F00101CE6B010ECD6F00014D
:107FF0000101CD510501FD5D0101CE510501FE5983
:108000000001D8A00EEF40F0010E24EC02F00101B7
:10801000CD2BD8B4CE2B0001D8A4E9D7939481847A
:108020000501FB51F35DFC51F4590001D8B01BEF81
:1080300040F0A5EC27F081A820EF40F03AEF41F0A6
:10804000010E80BAE86A356E010E81B6E86A351411
:10805000D8B42DEF40F0EFEF3DF0D8960501EEAB30
:10806000D8860001D8B652EF40F00101CE6B010E68
:10807000CD6F00010101CD510501FB5D0101CE5124
:108080000501FC590001D8A050EF40F0010E24EC8E
:1080900002F00101CD2BD8B4CE2B0001D8A4E9D732
:1080A000939281820501F951F35DFA51F45900016F
:1080B000D8B05DEF40F0A5EC27F081A862EF40F06A
:1080C0003AEF41F0010E80BAE86A356E010E81B6D2
:1080D000E86A3514D8B46FEF40F0AAEF3DF0D896B7
:1080E0000501EEADD8860001D8B694EF40F001014D
:1080F000CE6B010ECD6F00010101CD510501F95D7F
:108100000101CE510501FA590001D8A092EF40F0CB
:10811000010E24EC02F00101CD2BD8B4CE2B0001CE
:10812000D8A4E9D7939081800501F751F35DF85108
:10813000F4590001D8B09FEF40F0A5EC27F081A8DA
:10814000A4EF40F03AEF41F0010E80BAE86A356ED4
:10815000010E81B6E86A3514D8B4B1EF40F065EF8E
:108160003DF0D8960501EEAFD8860001D8B6D6EF1F
:1081700040F00101CE6B010ECD6F00010101CD5128
:108180000501F75D0101CE510501F8590001D8A0A4
:10819000D4EF40F0010E24EC02F00101CD2BD8B455
:1081A000CE2B0001D8A4E9D7949A828A0501F55113
:1081B000F35DF651F4590001D8B0E1EF40F0A5ECC1
:1081C00027F081A8E6EF40F03AEF41F0010E80BAC7
:1081D000E86A356E010E81B6E86A3514D8B4F3EF5B
:1081E00040F020EF3DF0D896060111A1D88600019D
:1081F000D8B618EF41F00101CE6B010ECD6F000132
:108200000101CD510501F55D0101CE510501F65980
:108210000001D8A016EF41F0010E24EC02F001019C
:10822000CD2BD8B4CE2B0001D8A4E9D7949882885E
:1082300081A81DEF41F03AEF41F005012B8DD89652
:10824000060111B7D8860001D8B629EF41F0A5EC98
:1082500027F0ABEF18F005012B9D0001ABEF18F0F4
:1082600005012B8D000181A838EF41F03AEF41F074
:10827000ABEF18F096EC2CF0ABEF18F0170EF76E92
:10828000580EF66E01EE31F001EC03F0D8A44CEF7D
:1082900041F0010E01016B6F0001170EF76E600EC9
:1082A000F66E01EE31F001EC03F0D8A466EF41F078
:1082B00001016B6B04EEA5F0170EF76E680EF66EFB
:1082C000D9EC02F0EF6A0001F9EC1EF01200170E73
:1082D000F76E7E0EF66E01EE31F001EC03F0D8A4DD
:1082E0007AEF41F006011187010E0101686F00016C
:1082F0008AEF41F0060111970101686B04EEA5F0C9
:10830000170EF76E820EF66ED9EC02F0EF6A0001DE
:10831000F9EC1EF01200170EF76E920EF66E01EEDB
:1083200031F001EC03F0D8A49BEF41F00601119766
:108330000101686B696B0001170EF76E980EF66EFF
:1083400001EE31F001EC03F0D8A4AEEF41F00601EC
:108350001187010E0101686F010E696F00011200A3
:1083600005EED1F011EE31F0060EE6CFEEFFE82E6D
:10837000FCD7EF6A04EEA5F0170EF76EA00EF66EAE
:10838000D9EC02F015EED1F0060EE75204E0E6CF8C
:10839000EEFFE82EFAD7EF6AF9EC1EF0120005EEB8
:1083A00093F015EED1F0060EE75204E0E6CFEEFFB3
:1083B000E82EFAD7EF6A9EEC2DF0120004EEA5F03D
:1083C000170EF76EB20EF66ED9EC02F011EE31F028
:1083D000360EE75204E0E6CFEEFFE82EFAD7EF6A5A
:1083E000F9EC1EF001EE31F084EC00F00501E06FD5
:1083F00021C0E1F50001120004EEA5F0170EF76EA2
:10840000C80EF66ED9EC02F011EE31F0360EE752DE
:1084100004E0E6CFEEFFE82EFAD7EF6AF9EC1EF0A3
:1084200001EE31F084EC00F00501E26F21C0E3F5CC
:10843000000112001FEC3AF004EEA5F0170EF76EE3
:10844000E00EF66ED9EC02F0020E016E0501ED5160
:10845000CCEC00F0EF6A0001F9EC1EF0120004EE23
:10846000A5F0170EF76EF80EF66ED9EC02F011EECD
:1084700031F0360EE75204E0E6CFEEFFE82EFAD7F1
:108480002E0EEE6EEF6AF9EC1EF001EE31F084EC88
:1084900000F00501ED6F0001120004EEA5F0180ECA
:1084A000F76E140EF66ED9EC02F011EE31F0360EC6
:1084B000E75204E0E6CFEEFFE82EFAD7200EEE6E8C
:1084C0006D0EEE6E730EEE6E2E0EEE6EEF6AF9EC22
:1084D0001EF001EE31F084EC00F00501F56F21C0D3
:1084E000F6F50001120004EEA5F0180EF76E2A0E44
:1084F000F66ED9EC02F011EE31F0360EE75204E0E0
:10850000E6CFEEFFE82EFAD7200EEE6E6D0EEE6E81
:10851000730EEE6E2E0EEE6EEF6AF9EC1EF001EEAB
:1085200031F084EC00F00501F76F21C0F8F500018F
:10853000120004EEA5F0180EF76E400EF66ED9ECA0
:1085400002F011EE31F0360EE75204E0E6CFEEFF16
:10855000E82EFAD7200EEE6E6D0EEE6E730EEE6EF6
:108560002E0EEE6EEF6AF9EC1EF001EE31F084ECA7
:1085700000F00501F96F21C0FAF50001120004EEC8
:10858000A5F0180EF76E560EF66ED9EC02F011EE4D
:1085900031F0360EE75204E0E6CFEEFFE82EFAD7D0
:1085A000200EEE6E6D0EEE6E730EEE6E2E0EEE6EF5
:1085B000EF6AF9EC1EF001EE31F084EC00F00501F9
:1085C000FB6F21C0FCF50001120004EEA5F0180EAF
:1085D000F76E6C0EF66ED9EC02F011EE31F0360E3D
:1085E000E75204E0E6CFEEFFE82EFAD7200EEE6E5B
:1085F0006D0EEE6E730EEE6E2E0EEE6EEF6AF9ECF1
:108600001EF001EE31F084EC00F00501FD6F21C099
:10861000FEF50001120004EEA5F0180EF76E820EB2
:10862000F66ED9EC02F011EE31F0360EE75204E0AE
:10863000E6CFEEFFE82EFAD7200EEE6E6D0EEE6E50
:10864000730EEE6E2E0EEE6EEF6AF9EC1EF001EE7A
:1086500031F084EC00F00601036F21C004F6000144
:10866000120004EEA5F0180EF76E960EF66ED9EC19
:1086700002F011EE31F0360EE75204E0E6CFEEFFE5
:10868000E82EFAD7200EEE6E6D0EEE6E730EEE6EC5
:108690002E0EEE6EEF6AF9EC1EF001EE31F084EC76
:1086A00000F00601056F21C006F60001120004EE7D
:1086B000A5F0180EF76EAA0EF66ED9EC02F011EEC8
:1086C00031F0360EE75204E0E6CFEEFFE82EFAD79F
:1086D000200EEE6E6D0EEE6E730EEE6E2E0EEE6EC4
:1086E000EF6AF9EC1EF001EE31F084EC00F00601C7
:1086F000076F21C008F60001120004EEA5F0180E65
:10870000F76EBE0EF66ED9EC02F011EE31F0360EB9
:10871000E75204E0E6CFEEFFE82EFAD7200EEE6E29
:108720006D0EEE6E730EEE6E2E0EEE6EEF6AF9ECBF
:108730001EF001EE31F084EC00F00601096F21C05B
:108740000AF60001120004EEA5F0180EF76ED20E24
:10875000F66ED9EC02F011EE31F0360EE75204E07D
:10876000E6CFEEFFE82EFAD7200EEE6E6D0EEE6E1F
:10877000730EEE6E2E0EEE6EEF6AF9EC1EF001EE49
:1087800031F084EC00F006010B6F21C00CF6000103
:108790001200310E0101315D0001D8A4D7EF43F082
:1087A0000501EE8901EEA0F0310EEE6EEF6A0001D8
:1087B000320E0101315D0001D8A4E6EF43F005015E
:1087C000EE8B01EEA0F0320EEE6EEF6A0001330E7A
:1087D0000101315D0001D8A4F5EF43F00501EE8DF4
:1087E00001EEA0F0330EEE6EEF6A0001340E0101CF
:1087F000315D0001D8A404EF44F00501EE8F01EED5
:10880000A0F0340EEE6EEF6A0001350E0101315D0D
:108810000001D8A413EF44F00601118101EEA0F08D
:10882000350EEE6EEF6A000104EEA5F0180EF76E3D
:10883000E60EF66ED9EC02F011EEA0F0140EE7523F
:1088400004E0E6CFEEFFE82EFAD7180EF76EEE0E34
:10885000F66ED9EC02F0EF6AF9EC1EF01200310E60
:108860000101315D0001D8A43DEF44F00501EE990E
:1088700001EEA0F0310EEE6EEF6A0001320E010142
:10888000315D0001D8A44CEF44F00501EE9B01EEF0
:10889000A0F0320EEE6EEF6A0001330E0101315D81
:1088A0000001D8A45BEF44F00501EE9D01EEA0F0BD
:1088B000330EEE6EEF6A0001340E0101315D0001EE
:1088C000D8A46AEF44F00501EE9F01EEA0F0340E4B
:1088D000EE6EEF6A0001350E0101315D0001D8A492
:1088E00079EF44F00601119101EEA0F0350EEE6E25
:1088F000EF6A000104EEA5F0180EF76EF80EF66EA2
:10890000D9EC02F011EEA0F0140EE75204E0E6CF2D
:10891000EEFFE82EFAD7190EF76E000EF66ED9ECC0
:1089200002F0EF6AF9EC1EF01200190EF76E0A0E53
:10893000F66E01EE31F001EC03F0D8A4A1EF44F0A3
:108940008288190EF76E0E0EF66E01EE31F001EC14
:1089500003F0D8A4ADEF44F0829882A8BBEF44F0B6
:1089600004EEA5F0190EF76E120EF66ED9EC02F0B9
:10897000EF6AF9EC1EF082B8C9EF44F004EEA5F0FE
:10898000190EF76E240EF66ED9EC02F0EF6AF9ECD0
:108990001EF01200190EF76E360EF66E01EE31F073
:1089A00001EC03F0D8A4D6EF44F0828A190EF76EDA
:1089B0003A0EF66E01EE31F001EC03F0D8A4E2EFCE
:1089C00044F0829A82AAF0EF44F004EEA5F0190E6A
:1089D000F76E3E0EF66ED9EC02F0EF6AF9EC1EF07F
:1089E00082BAFEEF44F004EEA5F0190EF76E500EB9
:1089F000F66ED9EC02F0EF6AF9EC1EF01200190ED7
:108A0000F76E620EF66E01EE31F001EC03F0D8A4C1
:108A10000BEF45F08180190EF76E660EF66E01EED3
:108A200031F001EC03F0D8A417EF45F0819081A05C
:108A300025EF45F004EEA5F0190EF76E6A0EF66EFE
:108A4000D9EC02F0EF6AF9EC1EF081B033EF45F09B
:108A500004EEA5F0190EF76E7C0EF66ED9EC02F05E
:108A6000EF6AF9EC1EF01200190EF76E8E0EF66E1C
:108A700001EE31F001EC03F0D8A440EF45F0818223
:108A8000190EF76E920EF66E01EE31F001EC03F066
:108A9000D8A44CEF45F0819281A25AEF45F004EE44
:108AA000A5F0190EF76E960EF66ED9EC02F0EF6A8D
:108AB000F9EC1EF081B268EF45F004EEA5F0190E56
:108AC000F76EA80EF66ED9EC02F0EF6AF9EC1EF024
:108AD0001200190EF76EBA0EF66E01EE31F001ECCF
:108AE00003F0D8A475EF45F08184190EF76EBE0E21
:108AF000F66E01EE31F001EC03F0D8A481EF45F001
:108B0000819481A48FEF45F004EEA5F0190EF76E65
:108B1000C20EF66ED9EC02F0EF6AF9EC1EF081B4E9
:108B20009DEF45F004EEA5F0190EF76ED40EF66E2B
:108B3000D9EC02F0EF6AF9EC1EF01200190EF76E94
:108B4000E60EF66E01EE31F001EC03F0D8A4ABEFC7
:108B500045F00601138F0001190EF76EEA0EF66E4E
:108B600001EE31F001EC03F0D8A4B9EF45F00601B5
:108B7000139F0001D896060113AFD8860001D8B61E
:108B8000CDEF45F004EEA5F0190EF76EEE0EF66E81
:108B9000D9EC02F0EF6AF9EC1EF0D896060113BF8B
:108BA000D8860001D8B6E0EF45F004EEA5F0190E26
:108BB000F76EFE0EF66ED9EC02F0EF6AF9EC1EF0DD
:108BC0000601118D000112001A0EF76E100EF66EDE
:108BD00001EE31F001EC03F0D8A4F1EF45F006010D
:108BE000148100011A0EF76E140EF66E01EE31F0CC
:108BF00001EC03F0D8A4FFEF45F006011491000149
:108C0000D896060114A1D8860001D8B613EF46F015
:108C100004EEA5F01A0EF76E180EF66ED9EC02F0FF
:108C2000EF6AF9EC1EF0D896060114B1D88600015F
:108C3000D8B626EF46F004EEA5F01A0EF76E280E11
:108C4000F66ED9EC02F0EF6AF9EC1EF00601118D18
:108C5000000112001A0EF76E3A0EF66E01EE31F0B8
:108C600001EC03F0D8A437EF46F0060114830001AD
:108C70001A0EF76E3E0EF66E01EE31F001EC03F0C7
:108C8000D8A445EF46F0060114930001D8960601DA
:108C900014A3D8860001D8B659EF46F004EEA5F02B
:108CA0001A0EF76E420EF66ED9EC02F0EF6AF9EC8E
:108CB0001EF0D896060114B3D8860001D8B66CEF22
:108CC00046F004EEA5F01A0EF76E520EF66ED9ECD1
:108CD00002F0EF6AF9EC1EF00601118D000112009E
:108CE000310E0101315D0001D8A47CEF46F082888D
:108CF000FA0E24EC02F08298320E0101315D00017F
:108D0000D8A488EF46F0828AFA0E24EC02F0829A08
:108D1000330E0101315D0001D8A494EF46F081804B
:108D2000FA0E24EC02F08190340E0101315D000155
:108D3000D8A4A0EF46F08182FA0E24EC02F08192D2
:108D4000350E0101315D0001D8A4ACEF46F08184FD
:108D5000FA0E24EC02F081940601118D000112003C
:108D600004EEA5F01A0EF76E640EF66ED9EC02F062
:108D7000EF6AF9EC1EF0010E0501ED6F010EEB6FCD
:108D8000F66B010EF56FF86B640EF76FFA6B640EFD
:108D9000F96FFC6B640EFB6FFE6B640EFD6F0601DA
:108DA000006B640E0501FF6F0601026B640E016F1C
:108DB000046B010E036F066B640E056F086B640E87
:108DC000076F0A6B640E096F0C6B640E0B6F0E6BF2
:108DD000640E0D6F106B640E0F6F1189118B0501FE
:108DE0002B85140E916F786BCD0E7C6FCC0E7B6F44
:108DF0004C0E7A6F7C0E796F0601119505014B6B55
:108E00004A6B496B486B4F6B4E6B4D6B4C6B536BA6
:108E1000526B516B506B576B566B556B546B01011A
:108E200069530001D8A417EF47F0E5EC4EF00101BB
:108E30006B6B686B060111970501266B5B6B5A6BB8
:108E4000596B586B5F6B5E6B5D6B5C6B636B626BDE
:108E5000616B606B676B666B656B646B6B6B6A6B8E
:108E6000700E696F830E686F6F6B6E6B700E6D6F37
:108E7000830E6C6F736B726B700E716F830E706FFD
:108E8000776B766B700E756F830E746F0401A46B35
:108E900001016C6B0501F46BFA0EF36F010E010119
:108EA000E16F010E0501D86F010ED96F010EDA6F67
:108EB000DB6BDC6BDD6BDE6B00011200010E05016C
:108EC000DF6FAA6AA96ADF51FEEC01F00A0E24ECFA
:108ED00002F0AA6A020EA96EE051FEEC01F0E15127
:108EE000FEEC01F00A0E24EC02F0AA6A040EA96E50
:108EF000E251FEEC01F0E351FEEC01F00A0E24EC2D
:108F000002F0AA6A060EA96EED51FEEC01F00A0EFF
:108F100024EC02F0AA6A0A0EA96E000EFEEC01F023
:108F2000AA6A140EA96EF551FEEC01F0F651FEECA2
:108F300001F00A0E24EC02F0AA6A160EA96EF7518F
:108F4000FEEC01F0F851FEEC01F00A0E24EC02F008
:108F5000AA6A180EA96EF951FEEC01F0FA51FEEC66
:108F600001F00A0E24EC02F0AA6A1A0EA96EFB5157
:108F7000FEEC01F0FC51FEEC01F00A0E24EC02F0D4
:108F8000AA6A1C0EA96EFD51FEEC01F0FE51FEEC2A
:108F900001F00A0E24EC02F0AA6A1E0EA96EFF511F
:108FA000FEEC01F006010051FEEC01F00A0E24EC8B
:108FB00002F0AA6A200EA96E0151FEEC01F00251E6
:108FC000FEEC01F00A0E24EC02F0AA6A280EA96E4B
:108FD0000351FEEC01F00451FEEC01F00A0E24EC0A
:108FE00002F0AA6A2A0EA96E0551FEEC01F00651A4
:108FF000FEEC01F00A0E24EC02F0AA6A2C0EA96E17
:109000000751FEEC01F00851FEEC01F00A0E24ECD1
:1090100002F0AA6A2E0EA96E0951FEEC01F00A5167
:10902000FEEC01F00A0E24EC02F0AA6A300EA96EE2
:109030000B51FEEC01F00C51FEEC01F00A0E24EC99
:1090400002F0AA6A320EA96E0D51FEEC01F00E512B
:10905000FEEC01F00A0E24EC02F0AA6A340EA96EAE
:109060000F51FEEC01F01051FEEC01F00A0E24EC61
:1090700002F0AA6A3C0EA96EE86A11B9010EFEEC74
:1090800001F00A0E24EC02F0AA6A3E0EA96EE86A0C
:1090900011BB010EFEEC01F00A0E24EC02F0AA6AEC
:1090A000400EA96E0401A451FEEC01F00A0E24EC5E
:1090B00002F0AA6A410EA96E05EED1F0EE5003E06F
:1090C000FEEC01F0FBD70A0E24EC02F001EECAF030
:1090D00015EED1F0010EF36E010EE1EC02F0EF6A35
:1090E000AA6A410EA96E01EECAF0EE5003E0FEEC52
:1090F00001F0FBD70A0E24EC02F001EECAF015EEE7
:10910000D1F0020EF36E010EE1EC02F0EF6AAA6AF2
:10911000420EA96E01EECAF0EE5003E0FEEC01F043
:10912000FBD70A0E24EC02F001EECAF015EED1F0E6
:10913000030EF36E010EE1EC02F0EF6AAA6A430E31
:10914000A96E01EECAF0EE5003E0FEEC01F0FBD791
:109150000A0E24EC02F001EECAF015EED1F0040E76
:10916000F36E010EE1EC02F0EF6AAA6A440EA96EFA
:1091700001EECAF0EE5003E0FEEC01F0FBD70A0E60
:1091800024EC02F001EECAF015EED1F0050EF36EFC
:10919000010EE1EC02F0EF6AAA6A450EA96E01EE3B
:1091A000CAF0EE5003E0FEEC01F0FBD70A0E24EC0F
:1091B00002F001EECAF015EED1F0060EF36E010ECC
:1091C000E1EC02F0EF6AAA6A460EA96E01EECAF05F
:1091D000EE5003E0FEEC01F0FBD70A0E24EC02F0A7
:1091E000AA6A500EA96EE86A0501EEB9010EFEECFE
:1091F00001F00A0E24EC02F0AA6A510EA96EE86A88
:10920000EEBB010EFEEC01F00A0E24EC02F0AA6A9D
:10921000520EA96EE86AEEBD010EFEEC01F00A0ED8
:1092200024EC02F0AA6A530EA96EE86AEEBF010EA2
:10923000FEEC01F00A0E24EC02F0AA6A540EA96EAC
:10924000E86A060111B1010EFEEC01F00A0E24ECF1
:1092500002F0AA6A550EA96E05019151FEEC01F0CB
:109260000A0E24EC02F0AA6A560EA96E7851FEECA2
:1092700001F00A0E24EC02F0AA6A570EA96E795189
:10928000FEEC01F07A51FEEC01F07B51FEEC01F0B6
:109290007C51FEEC01F00A0E24EC02F0AA6A5B0E8F
:1092A000A96EE86A060111B7010EFEEC01F00A0E84
:1092B00024EC02F0AA6A5C0EA96E05014851FEEC8E
:1092C00001F04951FEEC01F04A51FEEC01F04B5126
:1092D000FEEC01F00A0E24EC02F0AA6A600EA96E00
:1092E0004C51FEEC01F04D51FEEC01F04E51FEEC04
:1092F00001F04F51FEEC01F00A0E24EC02F0AA6AD4
:10930000640EA96E5051FEEC01F05151FEEC01F0DB
:109310005251FEEC01F05351FEEC01F00A0E24EC28
:1093200002F0AA6A680EA96E5451FEEC01F0555184
:10933000FEEC01F05651FEEC01F05751FEEC01F04D
:109340000A0E24EC02F0AA6A6C0EA96E01016851A3
:10935000FEEC01F00A0E24EC02F0AA6A6D0EA96E72
:109360006951FEEC01F00A0E24EC02F0AA6A6E0EBE
:10937000A96E6B51FEEC01F00A0E24EC02F0AA6A11
:109380006F0EA96E05015851FEEC01F05951FEEC2B
:1093900001F05A51FEEC01F05B51FEEC01F00A0EB7
:1093A00024EC02F0AA6A730EA96E5C51FEEC01F087
:1093B0005D51FEEC01F05E51FEEC01F05F51FEEC00
:1093C00001F00A0E24EC02F0AA6A770EA96E605131
:1093D000FEEC01F06151FEEC01F06251FEEC01F097
:1093E0006351FEEC01F00A0E24EC02F0AA6A7B0E37
:1093F000A96E6451FEEC01F06551FEEC01F066517E
:10940000FEEC01F06751FEEC01F00A0E24EC02F0D4
:10941000AA6A7F0EA96E6851FEEC01F06951FEEC5C
:1094200001F06A51FEEC01F06B51FEEC01F00A0E06
:1094300024EC02F0AA6A830EA96E6C51FEEC01F0D6
:109440006D51FEEC01F06E51FEEC01F06F51FEEC3F
:1094500001F00A0E24EC02F0AA6A870EA96E705180
:10946000FEEC01F07151FEEC01F07251FEEC01F0E6
:109470007351FEEC01F00A0E24EC02F0AA6A8B0E86
:10948000A96E7451FEEC01F07551FEEC01F07651BD
:10949000FEEC01F07751FEEC01F00A0E24EC02F034
:1094A000AA6A8F0EA96E01016C51FEEC01F00A0E42
:1094B00024EC02F0AA6A900EA96E05012651FEEC7A
:1094C00001F00A0E24EC02F0AA6A910EA96EF35183
:1094D000FEEC01F0F451FEEC01F00A0E24EC02F077
:1094E000AA6A930EA96E0101E151FEEC01F00A0E89
:1094F00024EC02F0AA6A940EA96E0501D851FEEC84
:1095000001F00A0E24EC02F0AA6A950EA96ED95158
:10951000FEEC01F00A0E24EC02F0AA6A960EA96E87
:10952000DA51FEEC01F00A0E24EC02F0AA6A970E62
:10953000A96EDB51FEEC01F00A0E24EC02F0AA6ADF
:10954000980EA96EDC51FEEC01F00A0E24EC02F03C
:10955000AA6A990EA96EDD51FEEC01F00A0E24EC08
:1095600002F0AA6A9A0EA96EDE51FEEC01F00A0E14
:1095700024EC02F0AA6A9B0EA96EE86A2BB5010ED4
:10958000FEEC01F00A0E24EC02F004EEA5F01A0E37
:10959000F76E8C0EF66ED9EC02F0EF6A0001F9EC72
:1095A0001EF01200000EF5EC01F00501DF6F020E57
:1095B000F5EC01F0E06FF7EC01F0E16F040EF5EC73
:1095C00001F0E26FF7EC01F0E36F060EF5EC01F04D
:1095D000ED6F0A0EF5EC01F0EB6FEB29EC6F140E5A
:1095E000F5EC01F0F56FF7EC01F0F66F160EF5EC07
:1095F00001F0F76FF7EC01F0F86F180EF5EC01F0E1
:10960000F96FF7EC01F0FA6F1A0EF5EC01F0FB6F51
:10961000F7EC01F0FC6F1C0EF5EC01F0FD6FF7ECC0
:1096200001F0FE6F1E0EF5EC01F0FF6FF7EC01F09C
:109630000601006F200EF5EC01F0016FF7EC01F070
:10964000026F280EF5EC01F0036FF7EC01F0046FE8
:109650002A0EF5EC01F0056FF7EC01F0066F2C0E09
:10966000F5EC01F0076FF7EC01F0086F2E0EF5EC4A
:1096700001F0096FF7EC01F00A6F300EF5EC01F024
:109680000B6FF7EC01F00C6F320EF5EC01F00D6F83
:10969000F7EC01F00E6F340EF5EC01F00F6FF7EC04
:1096A00001F0106F3C0EF5EC01F01189E8A0119962
:1096B0003E0EF5EC01F0118BE8A0119B400EF5EC8D
:1096C00001F00401A46F500EF5EC01F00501EE89E4
:1096D000E8A0EE99510EF5EC01F0EE8BE8A0EE9BC0
:1096E000520EF5EC01F0EE8DE8A0EE9D530EF5EC78
:1096F00001F0EE8FE8A0EE9F540EF5EC01F00601AC
:109700001181E8A01191550EF5EC01F00501916F62
:10971000560EF5EC01F0786F570EF5EC01F0796F0D
:10972000F7EC01F07A6FF7EC01F07B6FF7EC01F0EA
:109730007C6F5B0EF5EC01F006011187E8A0119734
:109740005C0EF5EC01F00501486FF7EC01F0496F94
:10975000F7EC01F04A6FF7EC01F04B6F600EF5EC9F
:1097600001F04C6FF7EC01F04D6FF7EC01F04E6F2C
:10977000F7EC01F04F6F640EF5EC01F0506FF7EC71
:1097800001F0516FF7EC01F0526FF7EC01F0536FFD
:10979000680EF5EC01F0546FF7EC01F0556FF7EC43
:1097A00001F0566FF7EC01F0576F6C0EF5EC01F01D
:1097B0000101686F6D0EF5EC01F0696F6E0EF5EC4E
:1097C00001F06B6F6F0EF5EC01F00501586FF7ECCF
:1097D00001F0596FF7EC01F05A6FF7EC01F05B6F95
:1097E000730EF5EC01F05C6FF7EC01F05D6FF7ECD8
:1097F00001F05E6FF7EC01F05F6F770EF5EC01F0B2
:10980000606FF7EC01F0616FF7EC01F0626FF7EC5D
:1098100001F0636F7B0EF5EC01F0646FF7EC01F083
:10982000656FF7EC01F0666FF7EC01F0676F7F0E84
:10983000F5EC01F0686FF7EC01F0696FF7EC01F0FF
:109840006A6FF7EC01F06B6F830EF5EC01F06C6F53
:10985000F7EC01F06D6FF7EC01F06E6FF7EC01F0D3
:109860006F6F870EF5EC01F0706FF7EC01F0716F20
:10987000F7EC01F0726FF7EC01F0736F8B0EF5EC03
:1098800001F0746FF7EC01F0756FF7EC01F0766F93
:10989000F7EC01F0776F8F0EF5EC01F001016C6FC2
:1098A000900EF5EC01F00501266F910EF5EC01F03C
:1098B000F36FF7EC01F0F46F930EF5EC01F001019A
:1098C000E16F940EF5EC01F00501D86F950EF5EC03
:1098D00001F0D96F960EF5EC01F0DA6F970EF5EC0A
:1098E00001F0DB6F980EF5EC01F0DC6F990EF5ECF2
:1098F00001F0DD6F9A0EF5EC01F0DE6F9B0EF5ECDA
:1099000001F02B85E8A02B95130EF65D0001D8A081
:1099100098EF4CF0D8A494EF4CF0890E0501F55D5A
:109920000001D8A098EF4CF00501F66B320EF56FF0
:10993000000101016B530001D8A4A1EF4CF0E5EC4C
:109940004EF001016B530001D8A4B2EF4CF004EECD
:10995000A5F01A0EF76EB20EF66ED9EC02F0EF6AB1
:10996000F9EC1EF0120004EEA5F01A0EF76EDA0EF6
:10997000F66ED9EC02F0EF6AF9EC1EF004EEA5F0F9
:109980001B0EF76E160EF66ED9EC02F0EF6AF9ECCC
:109990001EF004EEA5F01B0EF76E680EF66ED9EC05
:1099A00002F0EF6AF9EC1EF004EEA5F01B0EF76E64
:1099B000BA0EF66ED9EC02F0EF6AF9EC1EF004EE86
:1099C000A5F01C0EF76E020EF66ED9EC02F0EF6AEF
:1099D000F9EC1EF004EEA5F01C0EF76E4A0EF66EC2
:1099E000D9EC02F0EF6AF9EC1EF004EEA5F01C0EC3
:1099F000F76E880EF66ED9EC02F0EF6AF9EC1EF005
:109A000004EEA5F01C0EF76EC60EF66ED9EC02F051
:109A1000EF6AF9EC1EF004EEA5F01C0EF76EEE0EE8
:109A2000F66ED9EC02F0EF6AF9EC1EF004EEA5F048
:109A30001D0EF76E180EF66ED9EC02F0EF6AF9EC17
:109A40001EF004EEA5F01D0EF76E560EF66ED9EC64
:109A500002F0EF6AF9EC1EF004EEA5F01D0EF76EB1
:109A6000860EF66ED9EC02F0EF6AF9EC1EF004EE09
:109A7000A5F01D0EF76EBA0EF66ED9EC02F0EF6A85
:109A8000F9EC1EF004EEA5F01D0EF76EF00EF66E6A
:109A9000D9EC02F0EF6AF9EC1EF004EEA5F01E0E10
:109AA000F76E240EF66ED9EC02F0EF6AF9EC1EF0B8
:109AB00004EEA5F01E0EF76E6C0EF66ED9EC02F0F9
:109AC000EF6AF9EC1EF004EEA5F01E0EF76E900E94
:109AD000F66ED9EC02F0EF6AF9EC1EF004EEA5F098
:109AE0001E0EF76EB80EF66ED9EC02F0EF6AF9ECC6
:109AF0001EF004EEA5F01E0EF76EE00EF66ED9EC29
:109B000002F0EF6AF9EC1EF004EEA5F01F0EF76EFE
:109B1000320EF66ED9EC02F0EF6AF9EC1EF004EEAC
:109B2000A5F01F0EF76E700EF66ED9EC02F0EF6A1C
:109B3000F9EC1EF004EEA5F01F0EF76ED00EF66ED7
:109B4000D9EC02F0EF6AF9EC1EF004EEA5F0200E5D
:109B5000F76E180EF66ED9EC02F0EF6AF9EC1EF013
:109B600004EEA5F0200EF76E620EF66ED9EC02F050
:109B7000EF6AF9EC1EF004EEA5F0200EF76E920EDF
:109B8000F66ED9EC02F0EF6AF9EC1EF004EEA5F0E7
:109B9000200EF76ED00EF66ED9EC02F0EF6AF9ECFB
:109BA0001EF004EEA5F0210EF76E300EF66ED9EC25
:109BB00002F0EF6AF9EC1EF004EEA5F0210EF76E4C
:109BC000680EF66ED9EC02F0EF6AF9EC1EF004EEC6
:109BD000A5F0210EF76ED80EF66ED9EC02F0EF6A02
:109BE000F9EC1EF004EEA5F0220EF76E220EF66ED2
:109BF000D9EC02F0EF6AF9EC1EF004EEA5F0220EAB
:109C0000F76E600EF66ED9EC02F0EF6AF9EC1EF01A
:109C100004EEA5F0220EF76EC00EF66ED9EC02F03F
:109C2000EF6AF9EC1EF004EEA5F0230EF76E180EA5
:109C3000F66ED9EC02F0EF6AF9EC1EF004EEA5F036
:109C4000230EF76E560EF66ED9EC02F0EF6AF9ECC1
:109C50001EF004EEA5F0230EF76EA80EF66ED9ECFA
:109C600002F0EF6AF9EC1EF004EEA5F0230EF76E99
:109C7000FE0EF66ED9EC02F0EF6AF9EC1EF004EE7F
:109C8000A5F0240EF76E420EF66ED9EC02F0EF6AE4
:109C9000F9EC1EF004EEA5F0240EF76E880EF66EB9
:109CA000D9EC02F0EF6AF9EC1EF004EEA5F0240EF8
:109CB000F76EC60EF66ED9EC02F0EF6AF9EC1EF004
:109CC00004EEA5F0250EF76E120EF66ED9EC02F03A
:109CD000EF6AF9EC1EF004EEA5F0250EF76E500EBB
:109CE000F66ED9EC02F0EF6AF9EC1EF004EEA5F086
:109CF000250EF76E980EF66ED9EC02F0EF6AF9ECCD
:109D00001EF004EEA5F0250EF76EDA0EF66ED9EC15
:109D100002F0EF6AF9EC1EF004EEA5F0260EF76EE5
:109D20000E0EF66ED9EC02F0EF6AF9EC1EF004EEBE
:109D3000A5F0260EF76E460EF66ED9EC02F0EF6A2D
:109D4000F9EC1EF004EEA5F0260EF76E840EF66E0A
:109D5000D9EC02F0EF6AF9EC1EF004EEA5F0260E45
:109D6000F76EB60EF66ED9EC02F0EF6AF9EC1EF063
:109D700004EEA5F0260EF76EE80EF66ED9EC02F0B2
:109D8000EF6AF9EC1EF004EEA5F0270EF76E260E32
:109D9000F66ED9EC02F0EF6AF9EC1EF004EEA5F0D5
:109DA000270EF76E520EF66ED9EC02F0EF6AF9EC60
:109DB0001EF004EEA5F0270EF76E800EF66ED9ECBD
:109DC00002F0EF6AF9EC1EF0120004EEA5F0270E87
:109DD000F76EC40EF66ED9EC02F0EF6AF9EC1EF0E5
:109DE00001EE6DF0020E016E0501DF51CCEC00F0CA
:109DF000EF6A04EEA5F0270EF76EEC0EF66ED9ECC6
:109E000002F011EE6DF0320EE75204E0E6CFEEFF05
:109E1000E82EFAD7EF6A0001F9EC1EF001EE6DF0C2
:109E200015EEE4F0060EE75204E0E6CFEEFFE82E72
:109E3000FAD7EF6A04EEA5F0270EF76EFC0EF66E69
:109E4000D9EC02F011EE6DF0320EE75204E0E6CFED
:109E5000EEFFE82EFAD7EF6AF9EC1EF001EE6DF096
:109E6000020E016E086AE1C521F0E0C520F0CFECDA
:109E700000F0EF6A04EEA5F0280EF76E0C0EF66EF9
:109E8000D9EC02F011EE6DF0320EE75204E0E6CFAD
:109E9000EEFFE82EFAD7EF6AF9EC1EF001EE6DF056
:109EA000020E016E086AE3C521F0E2C520F0CFEC96
:109EB00000F0EF6A04EEA5F0280EF76E1C0EF66EA9
:109EC000D9EC02F011EE6DF0320EE75204E0E6CF6D
:109ED000EEFFE82EFAD7EF6AF9EC1EF001EE6DF016
:109EE000020E016E0501ED51CCEC00F0EF6A04EEBC
:109EF000A5F0280EF76E2C0EF66ED9EC02F011EEDE
:109F00006DF0320EE75204E0E6CFEEFFE82EFAD70E
:109F1000EF6A0001F9EC1EF001EE6DF0020E016E29
:109F2000086AF6C521F0F5C520F0CFEC00F0EF6A25
:109F300004EEA5F0280EF76E3C0EF66ED9EC02F09A
:109F400011EE6DF0320EE75204E0E6CFEEFFE82EA0
:109F5000FAD7EF6AF9EC1EF001EE6DF0020E016E19
:109F6000086AF8C521F0F7C520F0CFEC00F0EF6AE1
:109F700004EEA5F0280EF76E4C0EF66ED9EC02F04A
:109F800011EE6DF0320EE75204E0E6CFEEFFE82E60
:109F9000FAD7EF6AF9EC1EF001EE6DF0020E016ED9
:109FA000086AFAC521F0F9C520F0CFEC00F0EF6A9D
:109FB00004EEA5F0280EF76E5C0EF66ED9EC02F0FA
:109FC00011EE6DF0320EE75204E0E6CFEEFFE82E20
:109FD000FAD7EF6AF9EC1EF001EE6DF0020E016E99
:109FE000086AFCC521F0FBC520F0CFEC00F0EF6A59
:109FF00004EEA5F0280EF76E6C0EF66ED9EC02F0AA
:10A0000011EE6DF0320EE75204E0E6CFEEFFE82EDF
:10A01000FAD7EF6AF9EC1EF001EE6DF0020E016E58
:10A02000086AFEC521F0FDC520F0CFEC00F0EF6A14
:10A0300004EEA5F0280EF76E7C0EF66ED9EC02F059
:10A0400011EE6DF0320EE75204E0E6CFEEFFE82E9F
:10A05000FAD7EF6AF9EC1EF001EE6DF0020E016E18
:10A06000086A04C621F003C620F0CFEC00F0EF6AC6
:10A0700004EEA5F0280EF76E8C0EF66ED9EC02F009
:10A0800011EE6DF0320EE75204E0E6CFEEFFE82E5F
:10A09000FAD7EF6AF9EC1EF001EE6DF0020E016ED8
:10A0A000086A06C621F005C620F0CFEC00F0EF6A82
:10A0B00004EEA5F0280EF76E9C0EF66ED9EC02F0B9
:10A0C00011EE6DF0320EE75204E0E6CFEEFFE82E1F
:10A0D000FAD7EF6AF9EC1EF001EE6DF0020E016E98
:10A0E000086A08C621F007C620F0CFEC00F0EF6A3E
:10A0F00004EEA5F0280EF76EAC0EF66ED9EC02F069
:10A1000011EE6DF0320EE75204E0E6CFEEFFE82EDE
:10A11000FAD7EF6AF9EC1EF001EE6DF0020E016E57
:10A12000086A0AC621F009C620F0CFEC00F0EF6AF9
:10A1300004EEA5F0280EF76EBC0EF66ED9EC02F018
:10A1400011EE6DF0320EE75204E0E6CFEEFFE82E9E
:10A15000FAD7EF6AF9EC1EF001EE6DF0020E016E17
:10A16000086A0CC621F00BC620F0CFEC00F0EF6AB5
:10A1700004EEA5F0280EF76ECC0EF66ED9EC02F0C8
:10A1800011EE6DF0320EE75204E0E6CFEEFFE82E5E
:10A19000FAD7EF6AF9EC1EF0D8960501EEA9D88639
:10A1A0000001D8B6DFEF50F001EEA0F0280EF76EF8
:10A1B000DC0EF66ED9EC02F0EF6AE8EF50F001EE3B
:10A1C000A0F0280EF76EE60EF66ED9EC02F0EF6AFC
:10A1D00004EEA5F0280EF76EF20EF66ED9EC02F042
:10A1E00011EEA0F0140EE75204E0E6CFEEFFE82EE9
:10A1F000FAD7EF6AF9EC1EF0D8960501EEABD886D7
:10A200000001D8B60FEF51F001EEA0F0290EF76E65
:10A21000000EF66ED9EC02F0EF6A18EF51F001EE85
:10A22000A0F0290EF76E0A0EF66ED9EC02F0EF6A76
:10A2300004EEA5F0290EF76E160EF66ED9EC02F0BC
:10A2400011EEA0F0140EE75204E0E6CFEEFFE82E88
:10A25000FAD7EF6AF9EC1EF0D8960501EEADD88674
:10A260000001D8B63FEF51F001EEA0F0290EF76ED5
:10A27000240EF66ED9EC02F0EF6A48EF51F001EED1
:10A28000A0F0290EF76E2E0EF66ED9EC02F0EF6AF2
:10A2900004EEA5F0290EF76E3A0EF66ED9EC02F038
:10A2A00011EEA0F0140EE75204E0E6CFEEFFE82E28
:10A2B000FAD7EF6AF9EC1EF0D8960501EEAFD88612
:10A2C0000001D8B66FEF51F001EEA0F0290EF76E45
:10A2D000480EF66ED9EC02F0EF6A78EF51F001EE1D
:10A2E000A0F0290EF76E520EF66ED9EC02F0EF6A6E
:10A2F00004EEA5F0290EF76E5E0EF66ED9EC02F0B4
:10A3000011EEA0F0140EE75204E0E6CFEEFFE82EC7
:10A31000FAD7EF6AF9EC1EF0D896060111A1D8869B
:10A320000001D8B69FEF51F001EEA0F0290EF76EB4
:10A330006C0EF66ED9EC02F0EF6AA8EF51F001EE68
:10A34000A0F0290EF76E760EF66ED9EC02F0EF6AE9
:10A3500004EEA5F0290EF76E820EF66ED9EC02F02F
:10A3600011EEA0F0140EE75204E0E6CFEEFFE82E67
:10A37000FAD7EF6AF9EC1EF0D896060111A9D88633
:10A380000001D8B6D1EF51F004EEA5F0290EF76E1A
:10A39000900EF66ED9EC02F0EF6AF9EC1EF0DCEFED
:10A3A00051F004EEA5F0290EF76EA60EF66ED9EC6C
:10A3B00002F0EF6AF9EC1EF0D896060111ABD886D0
:10A3C0000001D8B6F1EF51F004EEA5F0290EF76EBA
:10A3D000BE0EF66ED9EC02F0EF6AF9EC1EF0FCEF5F
:10A3E00051F004EEA5F0290EF76ED40EF66ED9ECFE
:10A3F00002F0EF6AF9EC1EF004EEA5F0290EF76EFC
:10A40000EC0EF66ED9EC02F0020E016E05019151D0
:10A41000CCEC00F0EF6A0001F9EC1EF00501785376
:10A420000001D8A41DEF52F004EEA5F0290EF76E3E
:10A43000FC0EF66ED9EC02F0EF6A010E0501785DB4
:10A440000001D8A42DEF52F004EEA5F02A0EF76E0D
:10A45000140EF66ED9EC02F0EF6A020E0501785D7B
:10A460000001D8A44AEF52F004EEA5F02A0EF76ED0
:10A47000380EF66ED9EC02F0020E016E7CC52FF09C
:10A480007BC52EF07AC52DF079C52CF0030EFEECBD
:10A4900000F0EF6A01016C530001D8A45BEF52F0A9
:10A4A00004EEA5F02A0EF76E520EF66ED9EC02F00D
:10A4B000EF6AF9EC1EF0010E01016C5D0001D8A4F9
:10A4C0006DEF52F004EEA5F02A0EF76E660EF66EF2
:10A4D000D9EC02F0EF6AF9EC1EF001EE6DF0020E1D
:10A4E000016E5BC52FF05AC52EF059C52DF058C529
:10A4F0002CF0030EFEEC00F0EF6A04EEA5F02A0E3D
:10A50000F76E780EF66ED9EC02F011EE6DF0320EA9
:10A51000E75204E0E6CFEEFFE82EFAD7EF6AF9EC57
:10A520001EF001EE6DF0020E016E6BC52FF06AC5D4
:10A530002EF069C52DF068C52CF0030EFEEC00F07E
:10A54000EF6A04EEA5F02A0EF76E880EF66ED9ECCF
:10A5500002F011EE6DF0320EE75204E0E6CFEEFFAE
:10A56000E82EFAD7EF6AF9EC1EF001EE6DF0020E5C
:10A57000016E4BC52FF04AC52EF049C52DF048C5D8
:10A580002CF0030EFEEC00F0EF6A04EEA5F02A0EAC
:10A59000F76E980EF66ED9EC02F011EE6DF0320EF9
:10A5A000E75204E0E6CFEEFFE82EFAD7EF6AF9ECC7
:10A5B0001EF001EE6DF0020E016E5FC52FF05EC55C
:10A5C0002EF05DC52DF05CC52CF0030EFEEC00F006
:10A5D000EF6A04EEA5F02A0EF76EA80EF66ED9EC1F
:10A5E00002F011EE6DF0320EE75204E0E6CFEEFF1E
:10A5F000E82EFAD7EF6AF9EC1EF001EE6DF0020ECC
:10A60000016E6FC52FF06EC52EF06DC52DF06CC5B7
:10A610002CF0030EFEEC00F0EF6A04EEA5F02A0E1B
:10A62000F76EB80EF66ED9EC02F011EE6DF0320E48
:10A63000E75204E0E6CFEEFFE82EFAD7EF6AF9EC36
:10A640001EF001EE6DF0020E016E4FC52FF04EC5EB
:10A650002EF04DC52DF04CC52CF0030EFEEC00F095
:10A66000EF6A04EEA5F02A0EF76EC80EF66ED9EC6E
:10A6700002F011EE6DF0320EE75204E0E6CFEEFF8D
:10A68000E82EFAD7EF6AF9EC1EF001EE6DF0020E3B
:10A69000016E63C52FF062C52EF061C52DF060C557
:10A6A0002CF0030EFEEC00F0EF6A04EEA5F02A0E8B
:10A6B000F76ED80EF66ED9EC02F011EE6DF0320E98
:10A6C000E75204E0E6CFEEFFE82EFAD7EF6AF9ECA6
:10A6D0001EF001EE6DF0020E016E73C52FF072C513
:10A6E0002EF071C52DF070C52CF0030EFEEC00F0BD
:10A6F000EF6A04EEA5F02A0EF76EE80EF66ED9ECBE
:10A7000002F011EE6DF0320EE75204E0E6CFEEFFFC
:10A71000E82EFAD7EF6AF9EC1EF001EE6DF0020EAA
:10A72000016E53C52FF052C52EF051C52DF050C506
:10A730002CF0030EFEEC00F0EF6A04EEA5F02A0EFA
:10A74000F76EF80EF66ED9EC02F011EE6DF0320EE7
:10A75000E75204E0E6CFEEFFE82EFAD7EF6AF9EC15
:10A760001EF001EE6DF0020E016E67C52FF066C59A
:10A770002EF065C52DF064C52CF0030EFEEC00F044
:10A78000EF6A04EEA5F02B0EF76E080EF66ED9EC0C
:10A7900002F011EE6DF0320EE75204E0E6CFEEFF6C
:10A7A000E82EFAD7EF6AF9EC1EF001EE6DF0020E1A
:10A7B000016E77C52FF076C52EF075C52DF074C5E6
:10A7C0002CF0030EFEEC00F0EF6A04EEA5F02B0E69
:10A7D000F76E180EF66ED9EC02F011EE6DF0320E37
:10A7E000E75204E0E6CFEEFFE82EFAD7EF6AF9EC85
:10A7F0001EF001EE6DF0020E016E57C52FF056C52A
:10A800002EF055C52DF054C52CF0030EFEEC00F0D3
:10A81000EF6A04EEA5F02B0EF76E280EF66ED9EC5B
:10A8200002F011EE6DF0320EE75204E0E6CFEEFFDB
:10A83000E82EFAD7EF6AF9EC1EF005012653000165
:10A84000D8A42EEF54F004EEA5F02B0EF76E380EC0
:10A85000F66ED9EC02F0EF6AF9EC1EF0010E05017C
:10A86000265D0001D8A440EF54F004EEA5F02B0EB5
:10A87000F76E4E0EF66ED9EC02F0EF6AF9EC1EF0B0
:08A880001200B3EC4CF01200D1
:020000040030CA
:03000100861A0F4D
:020005008181F7
:060008000FC00FE00F40E5
:00000001FF
